:10000000980B0020E5000000C1000000C1000000C6
:1000100000000000000000000000000000000000E0
:10002000000000000000000000000000C10000000F
:100030000000000000000000C1000000C10000003E
:10004000492D0000F90500008D2E000079220000E6
:10005000F92100002D220000A52500006D260000DA
:10006000C1000000FD0100001D0200003D02000073
:100070001907000055460000C1000000C100000043
:10008000C1000000C1000000C1000000C10000006C
:10009000C1000000C1000000C1000000C10000005C
:1000A000C1000000C1000000C1000000C10000004C
:1000B000B12D0000D56B0000C1000000C1000000A0
:1000C000A02130B559251624054AC90588230120E9
:1000D0005560546053608B6803438B60F6E7C046FD
:1000E000FC000050002370B50A480B490B4C1A184D
:1000F0008A4203D2E55804331560F8E70021084B23
:10010000084A934201D202C3FBE704F01DFE00F04F
:100110002DFE70BD0000002000010020C86F00000F
:10012000000100209807002007B500230193032851
:100130001ED8114B02301B688000C340181C0723D7
:1001400018406B46033318701A78002A02D102F067
:100150003FFE04E01A78022A03D102F071FE0190FA
:1001600004E01B78072B05D1044B0193019802E0B2
:10017000034800E003480EBD140200500080510106
:100180000197FFFF0297FFFFF8B5071C0E1C01281F
:1001900015D9002913D00D1C0124381C291C06F088
:1001A00079FD084B821E9A4203D8013C2406204365
:1001B00007E080230134AD195B009C42EDD10120A2
:1001C0004042F8BDFDFFFF00094B40211A680A4379
:1001D0001A60084BC02292009858074901408020BD
:1001E000000201439950022200201A607047C04665
:1001F0000040004000E100E0FF00FFFF08B5054BB4
:1002000001219A680A439A60034B1869DB68984792
:1002100008BDC046200001400001002008B5054B84
:1002200001219A680A439A60034B586A1B6A9847EF
:1002300008BDC046000011400001002010B50D4B64
:1002400001219A680C4C0A439A60A36A5B18A36266
:10025000E36A002B0CD0236B002B09D0A36B013B6E
:10026000A363002B04D1E36B206C9847636BA363FB
:1002700010BDC0462000114000010020034B0122A8
:100280005A649A64DA641A657047C0460001002017
:10029000F0B585B003900C1C151C032800D97FE035
:1002A000434B06F0E3FC02213F585A6C012A79D1F6
:1002B000586D002876D13F495A658E6804273E4321
:1002C0008E603D4E3060B1680A43B260D866986572
:1002D0001C67FFF729FF211CFFF756FF03021B0ACB
:1002E000421C51D1354860E0986C01285AD15A6FB0
:1002F000002A57D12F4958678E6808273E438E60E1
:100300002F4E3260B1680143B1601A609A67DC67B2
:10031000FFF70AFF211CFFF737FF431CE2D003025F
:10032000FB4031E0DF6C0197012F3BD1254A11687A
:10033000002937D11F4E1760B06810273843B060CE
:10034000214E01983160B7683843B06051605961FF
:1003500094600220BDE71F6D0197012F22D119493A
:10036000CA68002A1ED1134ECF60B06820273843D8
:10037000B060164E01983260B7683843B0609A6238
:100380001A630C610320A4E77360000EEB061843A8
:100390003060022D08D103980F30C0B202F00CF883
:1003A0000B4802E00B4800E0002005B0F0BDC0465D
:1003B0000001002000020050000001400297FFFFF2
:1003C0002000014080010020000011402000114069
:1003D0000197FFFF0397FFFF73B50024032800D99F
:1003E000BDE0604C06F042FC02305E8B6069002884
:1003F00000D0B3E00125A561656901356561019013
:10040000019800282DDC019D1424654356484519A8
:10041000AD6D002D15D1019D012665434519AE65D1
:10042000019D65434519E965019D654345192966A7
:100430000199614341184A66019A54430019836641
:100440008AE001980130DAE7E069002800D085E011
:1004500001252562E5690135E561019001980028D3
:1004600001DD00247BE0019D142465433E482D58A6
:10047000002D14D1019D012665432E50019D654339
:1004800045196960019D65434519A960019961435A
:100490004118CA60019A5443001903615CE0019855
:1004A0000130DAE7606A002858D10125A562656A43
:1004B00001356562019001980028D2DC019D142469
:1004C0006543294845196D69002D15D1019D012607
:1004D000654345196E61019D65434519A961019DFB
:1004E00065434519E9610199614341180A62019A1E
:1004F0005443001943622FE001980130DAE7E56ABE
:10050000002D2BD118480126C662E66A0136E66244
:10051000019502E0019C01340194019C002CA0DCB7
:10052000019D1424654345192D6B002DF2D1019DC9
:100530000126654345192E63019D6543451969638D
:10054000019D65434519A963019961434118CA6337
:10055000019A544300190364019C00E0034C201CE1
:1005600076BDC04680010020000100200497FFFFF7
:1005700030B503281FD8114B8200D358104A0830D9
:100580009B181968802292050A431A60C0B20D4B6D
:10059000C2220321920001409C58C900FF258D40D2
:1005A000AC4380258D40291C214399500122824073
:1005B0001A60002000E0044830BDC046806F000093
:1005C0000000014000E100E00197FFFF03280BD885
:1005D000064B8000C358064A00209B1819688022E9
:1005E000D2050A431A6000E002487047806F00009D
:1005F000000001400197FFFF084B07B51A6808216A
:100600009206D20F01921A680A431A60044B1B6BC0
:10061000002B01D00198984707BDC046004000401C
:10062000800100200C4B01225B68134212D00B4B5F
:1006300099680A439A600A4B80211A688A431A60B3
:10064000072210400202074918680840104318604A
:10065000002000E004487047FC00005000020050F9
:1006600000400040FFF8FFFF0697FFFF034B4021CB
:100670001A680A431A60024B186370470040004032
:100680008001002008B509283CD806F0EFFA0509DA
:100690000D10191E22262A311B4B80211A6812E0E8
:1006A000194B80211A681FE0FFF78EFD2BE0164BD7
:1006B00040211A688A431A60144B0222DA6715E057
:1006C000114B10211A680A430FE00F4B10211A68D2
:1006D0000AE00D4B01211A68F5E70B4B02211A685D
:1006E000F1E7094B02211A688A431A6000200AE0E8
:1006F000054B072211400A021868054901401143C1
:100700001960F3E7034808BD0040004004E100E041
:10071000FFF8FFFF0597FFFF044B10B51868044B67
:100720001B68002B00D0984710BDC0461C00054038
:10073000B4010020824BF7B50D00184200D0F3E061
:100740008A79072A00D9F1E0AB23D340DB0700D434
:10075000ECE00B79032B00D9EAE04B79012B00D9AF
:10076000E8E0CB79062B00D9E6E0A023DB0575494C
:10077000DA688024002805D164022243DA60DE684A
:10078000714A04E0A4022243DA60DE686F4A324014
:10079000DA608B680F2623438B606D4BC4180420EE
:1007A000A3680343A3600223A2681A43A260EF79FF
:1007B000A2683E40F0278640BA433243A260AE7939
:1007C000D03F0640721E9641E2687601BA4332433A
:1007D000E260AA79E76813405A1E93411A01102378
:1007E0009F433B00012608271343E360AA79E3688F
:1007F0003240D200BB431343E360E3682A79053FEC
:100800003A40BB431343E360E2686B7982431E4086
:10081000B30016001E43E660236A2A7AFB30834346
:10082000134323620A68474BD20703D55869494AE4
:1008300002400FE01A6AD20305D45869454A0240C3
:100840008020400405E01A68520777D5C0205A6915
:10085000800402435A618E694B693605360F9B014D
:100860009B0F0136002B02D102F0B2FA07E0354BA4
:100870005B699B019B0F012B03D102F0ADFA3100A4
:1008800001E03100344806F005FA2F68060039000F
:1008900006F000FA0F2305000340626A012B0CD812
:1008A0007F01B74209D22D4B050913406362626A8A
:1008B0002B4BAF1E134063622EE0802180238905FD
:1008C0000A436262626A5B051A43264BAF1E62628C
:1008D0009F4221DD0826636A0B436362626A204BF4
:1008E00013406362731C19002800019306F058FA44
:1008F00002290ED80F23616A1B4A1E40114033069D
:100900000E001E4366620199280006F0C3F9871E97
:1009100002E0019E102EE5D1656AB8B22D0C2D04BF
:100920000543656200200AE0104808E0104806E030
:10093000104804E0104802E0104800E01048FEBDF6
:10094000FFFFEFFF00020050FFFFFEFFFFFFFDFF74
:1009500000000540FFFFFFFC00805101FFFFFFDFAB
:10096000FFFFFFEFFFFF0000FFFFFFF00298FFFF18
:100970000398FFFF0498FFFF0598FFFF0698FFFF0D
:100980000898FFFFF7B501240E002E4B0192C31803
:100990005D682640A54335434E0802272640A64001
:1009A0005D605D68BD4335438E082640BE405D6096
:1009B0005D68FF19BD4335435D605D68CE08264024
:1009C0000437F600BD4335435D605E680D09B446EB
:1009D00062461D4E2540EF0216403E4310275E60E2
:1009E0005E682D01BE4335434E09890926400C40FF
:1009F000A10140245D605D68FF197601BD43354368
:100A00005D605D68A5432C000C43C3215C608900D8
:100A10000E4B00280BD1019A0D480260FF205A5856
:100A200082437F3802435A508022520108E05858CE
:100A3000084A02408020000202435A50802292015C
:100A40001A60F7BD00000540FFF7FFFF00E100E07E
:100A5000B4010020FF00FFFF0322F0B5214B224E1E
:100A6000C018036B214F134303634C780123621EAC
:100A70009441C56A1E4AE4032A402243C262C56A01
:100A80008A7814062A02120A2243C2620C78C26AC9
:100A90001C40324024022243C2620C78C26ADC400D
:100AA000144D1C4064022A402243C2620C78C26A80
:100AB000A4081C40A4023A402243C262076ACC78D0
:100AC0000D4A24023A40224302620A7981681340A7
:100AD0001A020B0033401343836003691D40056114
:100AE000F0BDC04600000540FFFEFFFFFFFBFFFF1B
:100AF000FF7FFFFFFFFDFFFFFF00FFFF30B5124B41
:100B00000F22DC681025944301221443DC60DC686A
:100B1000AC43DC60DC6820252C43DC6058609960C5
:100B200019690A431A61BFF36F8F18690121064AD8
:100B30000840FAD113689B090B4204D01368402186
:100B40000B430248136030BD00C000508188FFFF96
:100B500010B5144B0F24DA68A243DA60DA68102467
:100B6000A243DA60DA682024A243DA6000225860E7
:100B70009A601A69012002431A61BFF36F8F1869E6
:100B80000124084A2040FAD113689B09234205D06A
:100B9000136840210B431360034801E092680A6028
:100BA00010BDC04600C000508188FFFF124B0F21CE
:100BB000DA688A4302210A43DA60DA6810218A433C
:100BC000DA60DA6820210A43DA6058601A69012184
:100BD0000A431A61BFF36F8F18690121064A084062
:100BE000FAD113689B090B4204D0136840210B43D0
:100BF000024813607047C04600C000508188FFFF64
:100C0000054B04215A680A435A60044B01211A68B3
:100C10000A431A607047C0460002005000C00050EE
:100C2000024B01211A688A431A60704700C00050C5
:100C300010B5162059248821034B5C605860596018
:100C40005A68002AF9D010BDFC000050F0B50C0025
:100C500085B0FF2813D102213D4A93680B4393606E
:100C6000FFF7E6FFFFF7CCFFF8204002FFF79EFFFB
:100C7000A0220121D20593680B439360FEE7013067
:100C8000C5B2FF20152D60D8012D0ED1092905D937
:100C90000B1C182900D91823DCB200E00A242D4BC4
:100CA0001B190A3B1A782C4B1A602C4B585D019388
:100CB000C0B2844249D0FFF7BBFF8022284B92018B
:100CC000DA67FFF79DFFF823DB01EE18B60003A9F2
:100CD0003000FFF73DFF039B102723409C4209D1C2
:100CE000204B3000E1180391FFF708FF1EE0013FA1
:100CF000002F1BD0F8204002FFF758FFF82003A96F
:100D00004002FFF725FF039B0133F0D1019B5C55A7
:100D10000024019B195D134BC918F823DB01E0186F
:100D200080000134FFF7EAFE152CF2D103A9300050
:100D3000FFF70EFF039BDCB2FFF772FF80220A4B26
:100D400092011A6001F0ECFF200005B0F0BDC04632
:100D500000410050906F000010000440EB020020A2
:100D600004E100E00000FFFF00E100E0F0B5594BB6
:100D7000594F5A4A3B605A4B5A4E1A605A4A5B4D79
:100D800032605B4A5B4C2A605B4AF9B02260802289
:100D9000B2600022BA609A600A23AB602E33A3606F
:100DA000FFF746FF0121554B1A680A431A6008975E
:100DB0001F00039605950794FB68504ADB07FBD597
:100DC000116A4F4B4F4C0B4013620C2301212360DF
:100DD000BC3322681A430A4204D122685B085208D5
:100DE0002260F6E7C02122680902023A5202386AFC
:100DF0000A43023B1343DA05400A4002D20D024384
:100E00003A62F8229201386A13403F4A0240134383
:100E10003B623B6A194339623A6A3C4B13403B627E
:100E20003B6A3B4A13403B620E92FB68334A5B07C6
:100E3000FBD5072113698B4305390B431361D36835
:100E40001B0603D5D3687E310B43D36003F038FF14
:100E500001F0C2FF2060FFF7D3FEF82012A9400284
:100E6000FFF776FE2B4B129A2B4C9A4211D100259C
:100E7000F823DB01E818800012A9FFF769FE129B36
:100E8000DBB263550135152DF2D1F925234E6D02E4
:100E90004CE012A92248FFF75BFEF820129B4002AB
:100EA000DBB223750025FFF781FE142D03D01D4B07
:100EB0000F33EB5C6355615D1B4BC918F823DB01F5
:100EC000E818800001351291FFF718FE152DECD1BE
:100ED000DBE7C046FFCF000000400050F0FF0000FD
:100EE0004040005080400050FFF70000C0400050DC
:100EF000CF5D000000410050D50F000000020050FF
:100F0000FFFFF7FFD0020020FFC1FFFFFFFFFBFF45
:100F1000FFFFFEFFA500FFFFEB0200204F050020B2
:100F200050F00100906F00000000FFFF12A92800A0
:100F3000FFF70EFEF54B129AE918F54B100E5854B8
:100F4000110C3170B270110AF24A04357170043616
:100F50009542EBD11A78FF2A03D1DF3A1A700022AA
:100F60005A7012A9EC48FFF7F3FDFFF759FE002075
:100F700092210126E94BEA4A1870129B09061B02CE
:100F80001B0A13601368E74D5B181360E64B83225E
:100F90001E70032302210093030005F0C3FD6A6A5B
:100FA000E24B13408022920013436B62E04B1E60C1
:100FB00005F04AFE059B1B6902959B0701D404239B
:100FC0002371079B1B691B0703D404226379934396
:100FD0006371079B1B69DB0607D4082263791343FF
:100FE00063716379043A93436371079B1B699B06A2
:100FF00007D408226379934363716379043A1343F6
:10100000637163791B0705D54022039B9B681343DB
:10101000039A936090220025039BA0249B68E4051B
:101020001343039AC34E9360C34BC44A1D70C44B11
:101030001D70BB4B1B68DBB21370C24A13701F23B9
:1010400011780B401370C04AC04B11680B4003214C
:101050000B431360BE4ABF4B11680B40C02109010E
:101060000B4380211360E26849020A43E260E268B0
:101070000E9B1A40E260BB680B430421BB60B64B79
:101080009A680A439A609A6802390A439A609A6891
:10109000EE318A439A60DA68D0398A43DA60DA68D6
:1010A0001D390A43DA60DA6801318A43DA60DA68A6
:1010B0008A43DA601A6AFB318A431A627A69A74B5B
:1010C00013407B61BB691B051B0F049301F080FE7D
:1010D00080223368920513438022336033685205BF
:1010E00013433360049B591C05F0D4FD9C4905F063
:1010F000D1FD3268023883B2100C0004184330600E
:10110000226B984BC326134008222363236B0121D3
:1011100093432363236B944A280013402363236B78
:10112000B60013402363914AFFF72CFCFF22904C3A
:101130001420A35993437F3A1343A35101F03CF980
:101140008C498D4B0A220B6003230B7101238020F5
:101150004D718B71724BCD711B6840031343DBB231
:101160000B72FFF7E7FA012310A980204B700523CB
:1011700040030B708D70CD700D71FFF76DFC8020FA
:101180002A0001214003FFF7FDFBA3597B4A2900F8
:1011900013408022D2011343A351062001F094F89A
:1011A0000221032001F076F80321080001F072F813
:1011B000734B0D201D7001F0FFF80E2001F0FCF8BC
:1011C000059A704B0C3ED3610523059A5B429361EF
:1011D00009332360A3596C4A01211340A3512A000B
:1011E0006A4B032001F08AF8C022A35912061B02A1
:1011F0001B0A1343A35101F09DFA152001F0DCF8FE
:10120000012314AE3370624B29001593322328005A
:1012100016937570179501F059FD3100280001F003
:10122000F7FA0121280001F0FFFC0121280001F05C
:1012300099FA4D4B574A51780F93534B04940693A8
:10124000534B0B932B00092906D951780E331829DB
:1012500002D853780A3BDBB200244F4A0125D25C06
:101260004E4B4F4E1A604F4B1C70FFF707F8202271
:10127000BB684D491343C022BB603460B368802013
:101280002B43B360716033685205944613430422C4
:1012900033603368C00503433360BB681343BB60EE
:1012A000424B1C609A682A439A60624659601968EA
:1012B00011431960FA211A68890002431A60280054
:1012C0002A00FEF7E5FF2800FFF780F92800FFF766
:1012D0004FF92300364A29002800FFF77DF8C22283
:1012E000049B92009B58254AC2211340C02212023F
:1012F0001343049A89005350022022002D49FEF71F
:10130000C7FF0220FFF734F956E0C046000EFEFF8B
:101310004E05002018F20100FC0F1000B002002062
:10132000B802002000000E4016030020FFFCFFFF63
:101330001C000050240005409407002044050020B4
:10134000B40200203D0400203C000050FCFCFFFFE4
:1013500030000050F3F3FFFF00000540FFFFFFFCEB
:1013600090D00300FFF7FFFFFFFBFFFFA145000048
:1013700000E100E0D402002020A10700FF00FFFFF1
:101380007205002004000400FFFF00FFE1320000AE
:1013900030750000EB020020906F00001000044048
:1013A0002000114076050020FFFF000000000140F2
:1013B000C9330000F82A00002300CA4A290002208D
:1013C000FFF70AF8C222049B92009B58C64AC2212A
:1013D0001340C02212041343049A89005350200082
:1013E000290001F0C1FC03227B69062013437B61C5
:1013F000FFF718F9BD48FFF739F921000220FFF780
:1014000041F921002000FFF73DF901F089FCB84BBC
:1014100009961C70B74B1C80B74B1B78A34204D0B5
:101420008023B64A1370B64B1D70002301270A9320
:101430000C93049380330693FFF7FAFBB14A1368C9
:101440003B43136001F06CFCAC4B1B785BB2002B90
:1014500003DBFA22AC4B52001A60AC4B1B685B07F3
:1014600028D5FFF7E5FBFFF7CBFBF920F924400275
:10147000FFF79CFBA64D6402A64BA74AE318D15C7C
:101480002B7809061B04C9186B7820001B02C918A9
:10149000AB780434C918FFF731FBA04B04359C42EC
:1014A000EAD1FFF7BDFB01F03BFC0421974A13682A
:1014B0008B4313609A4B1A68920541D51968994A73
:1014C0000A401A608D4A9849127852B2002A01DA0D
:1014D000052200E000220A700021944A944C1180F9
:1014E0001B682178C9B29B0211D408250A20FFF796
:1014F000ADFB23788F4CDBB28F4EE37231780B203B
:101500002943FFF7A3FB33781D43257313E0082617
:101510000C20FFF79BFB2378864D874CDBB26B7367
:1015200023780D20BB43237021783143FFF78EFBD6
:1015300023781E43AE737A4A804B11680B401360C8
:101540007F4B1B78032B00D024E27E4B1A787E4B16
:101550001B789A4258D1802371499B040C681C4027
:1015600054D16A4B1A68520350D51A683A424DD08A
:101570001A68BA431A60754B1B78002B46D080223C
:1015800006250B68D20413430B60714B1878C0B268
:10159000421CD2B21A706F4A15541878C0B2451C5A
:1015A000EDB21D70052515541878C0B2451CEDB27A
:1015B0001D7014541878C0B2441CE4B21C70664C00
:1015C000A44666462478E4B2651CEDB23570145426
:1015D0001878C0B2441CE4B21C70862414541878E5
:1015E000C0B2441CE4B21C70042414541878C0B275
:1015F000441CE4B21C70554B1B78DBB213540A68D0
:10160000564B13400B6001E003F0ECFB3F4B1B68B3
:101610005B0300D437E18020414BC00419680140CE
:1016200000D030E11A6802431A601A68120200D42E
:10163000EAE018684A4A02401A60304B1B785BB2F5
:10164000002B00DB90E020220A24039B424E9B6883
:101650009343039A93603E4B1878C0B2421CD2B2B7
:101660001A703C4A14541878C0B2441CE4B21C707E
:10167000092414541878C0B2441CE4B21C701154EC
:101680001878C0B2441CE4B21C703478E4B2651C13
:10169000EDB23570145418783025C0B2441CE4B251
:1016A0001C70B22414541878C0B2441CE4B21C70EC
:1016B00017541878C0B2441CE4B21C706C4664190C
:1016C000247814541878C0B2441CE4B21C7011542D
:1016D0001978C9B2481CC0B2187022480078C0B24C
:1016E000505482E0F5390000FFFF00FFB54C0000C8
:1016F0002603002074050020160300207605002034
:101700006605002000400040E00200208007002025
:101710004F050020000EFEFF4E05002018F20100CC
:101720006C050020FFFDFFFFB0020020B202002088
:1017300027030020EB0200207C070020FFFFCFAF33
:1017400094070020950700208807002084070020C8
:10175000EA0200203F04002040050020FFFFFFFBBD
:10176000FFFF7FFF150300200A24BE4BBE4E1878F2
:10177000C0B2421CD2B21A70BC4A14541878C0B21B
:10178000441CE4B21C70092414541878C0B2441CE0
:10179000E4B21C7011541878C0B2441CE4B21C703E
:1017A0003478E4B2651CEDB2357014541878C0B2C8
:1017B000441CE4B21C70B22414541878C0B2441C07
:1017C000E4B21C7017541878C0B2441CE4B21C7008
:1017D00011541878C0B2441CE4B21C70115418782B
:1017E000C0B2441CE4B21C7011541978C9B2481C30
:1017F000C0B21870022050541978C9B2481CC0B247
:1018000018706B461B7C5354994B9A491A685201C5
:1018100035D505241A68944E0A401A60914B187801
:10182000C0B2421CD2B21A70904A14541878C0B296
:10183000441CE4B21C70042414541878C0B2441C34
:10184000E4B21C70002414541878C0B2441CE4B2F2
:101850001C703478E4B2651CEDB2357014541878FD
:10186000C0B2441CE4B21C70B02414541878C0B246
:10187000441CE4B21C70804B1B78DBB213547F4BCA
:101880001A68114019607C48069A03789A4200D180
:10189000BFE00378764A5BB2002B47DB0378DBB20C
:1018A000069313685B0300D4B3E0802205257349D7
:1018B000D2040B6813430B606A4B1C78E4B2621CC1
:1018C000D2B21A70694A15551C78E4B2651CEDB2A3
:1018D0001D70042515551C78E4B2651CEDB21D7011
:1018E000002515551C78E4B2651CEDB21D705E4DE7
:1018F0000D94AC4664462D78EDB26E1CF6B226709F
:101900000D9C15551C78E4B2651CEDB21D70B02518
:1019100015551C78E4B2651CEDB21D700378DBB27E
:1019200013550A68534B13400B6072E02021039B50
:1019300040249B688B4303998B608021099BC904D9
:101940001B680B4309990B608021099BC9051B6823
:101950000B4309990B608021089B9B680B430899F6
:101960008B60059B05999B68A3438B60444BD9789A
:10197000444B49001980FA2113684900234313603E
:10198000414B196000231C0018A95C520233802BC4
:10199000FAD183E7384A06991378994239D01378F7
:1019A0005BB2002B32DA394B1B88002B31D120215E
:1019B000039B9B688B4303998B600421059B3448F0
:1019C0001B690B40FAD18024089989682143089C3F
:1019D000A16040248168A143816002200799896841
:1019E00081430798816026492648C97849000180CB
:1019F0001F4801682143016019001278D2B2069293
:101A000018AA99520233802BFAD102E01378DBB284
:101A10000693204B1A88002A00D18EE200221A80F9
:101A2000029A1D4B126BD20700D486E21A6B104C3F
:101A30003A431A632168194AC90331D419688903E2
:101A400004D5117818684B0018A9C852029B5B682E
:101A50009B0329D51049137849685B0058A8C152E7
:101A600022E0C046EA020020400500203F0400209A
:101A700080070020FFFFFFFB760500206C0500209B
:101A8000EB020020A4020020E0020020E40200207B
:101A9000C04000504205002000000E4026030020F8
:101AA00023680E990B402360029BDB699B0309D5D9
:101AB000137838A8DBB2591CC9B21170D0495B0049
:101AC000C969C1523F2311780B401370FA22029B5F
:101AD00012011B689BB2934200D8DCE0C94B1B7813
:101AE0005BB2002B00DBD6E0202240202368C649F1
:101AF000134323608A78C54B1A80226802420BD0B8
:101B0000226882432260CA78198852008A1892B2E9
:101B10001A800022BE4B1A8080214020BD4A936863
:101B20008B439360BC4B9968014399603C381D69B5
:101B3000B9490542FBD18025906828439060402038
:101B40008A6882438A60B54A1288002AFBD0002145
:101B50000720B24A1180B2490A68824380203A4382
:101B60000A60029A0001126A024302980262029815
:101B7000A34A006BC007FAD50025106B38431063E9
:101B8000A84805701068A84D80B2A84204D99F4AA1
:101B90001288002AC0D12BE007260868B0438026AF
:101BA00038430860106A3601304310620298944A44
:101BB000006BC007FAD5106B38431063106880B211
:101BC000A842E4D807260868B0433843086080205C
:101BD000116A000101431162106B8949C007FBD5EE
:101BE0000A6B3A430A630A6892B2AA42CFD852E01B
:101BF000FA21029A0901126892B28A424BD98021D5
:101C0000844A80209268C0038A438249874D8A6053
:101C100040219A680A439A60854A3D391170794A91
:101C20001770844A116801438348116001780131BB
:101C3000C9B2017081490D8006787349804D052E27
:101C40000AD98E7A002E01D0897A00E0497AC9B289
:101C500029700021017002E0497AC9B22970002080
:101C6000784908801068784901401160774A1188E6
:101C7000002910D120207649118076498A680243D4
:101C80008A602268520306D510219A680A439A6036
:101C90001422714B1A602022072123689343604A63
:101CA000236013688B433B4313608022029B120125
:101CB0001B6A1343029A136200231A00180018A922
:101CC000595A0D1C914200D2151CAAB29508A9427E
:101CD00001D2801800E040180233802BEFD13E2162
:101CE00004F0D8FF484DC3B20A932B7D984201D22D
:101CF000287DC0B22B7D6421C01AAF235B005843FE
:101D000004F0C8FF554B1A68801840081860FA2381
:101D10002A799B005343434A984201D2002313700F
:101D200023685B0601D5002313708023394E316987
:101D30000B4000D11370A9781378994249D200233F
:101D40001370802240218020B368C0039343B360A6
:101D5000314B9A680A439A60354A3D391170294AD5
:101D60001770344A11680143116033490878013013
:101D7000C0B208702D4884466346304803800B7813
:101D80002F48052B05D90023AD7AEDB205700B70F5
:101D900002E0697AC9B2017000202A4908801068FF
:101DA000294901401160294A1188002911D12020B8
:101DB0002749118027498A6802438A6022685303B1
:101DC00007D51021144B9A680A439A601422224BBB
:101DD0001A60224B224A1B680F2B49D9CF2B02D8FD
:101DE0009B080C3344E01F498B4202D81B09333354
:101DF0003EE01D498B4239D89B096C3338E0C04620
:101E000000000E4076050020EB0200209207002023
:101E1000A402002000400050C040005042050020B5
:101E200030000E404D0500209F0F00008813000079
:101E3000B00200206C0500204C0500202403002087
:101E40006A050020B2020020FFFFFFBFBE02002093
:101E5000DC0500008040005048050020B80100204B
:101E600015030020FF040000FF1400001B0A553B6F
:101E700000242000DBB2137038ABE35A0234C018E0
:101E8000802CF9D1CE4B80095843CE4B000B9842A1
:101E90002AD864235B425843CB4BAF21C01804F0CF
:101EA000F9FEC3B20493502B20D9B368C748A343AB
:101EB000B360C74B403C9A6822439A60022202708A
:101EC0009968214380249960C24BE400196821433A
:101ED0001960C1490A7000210270C04A1180196856
:101EE000BF4A0A401A6016E000230493B94B1A68EF
:101EF000520510D5049A402A0DD81A680F990A4045
:101F00001A600022B44B1A70B64B1978AF4B0329F4
:101F100000D106321A700022130058A811007E3139
:101F2000415A023A5B1811007E31F7D1FA229B091F
:101F3000520053431B0BDBB20C93A64803683B4291
:101F400001D1FFF779FA0F21A74B1A788A43C02AEB
:101F50000ED19A78D2B25A70DA78D2B29A701A79CF
:101F6000D2B2DA705A79D2B21A719A79D2B25A715F
:101F70000F215A788A43E02A00D01AE15978D43ADE
:101F80000A400C2A00D014E18025924A5C789978A6
:101F90001668ED05E4B2C9B22E4200D1F6E0DB7856
:101FA0003E2B09D00521894B197000218B4B1980DC
:101FB00011688B4B0B4013608B4AD378DBB2382B04
:101FC00000D1A3E037D82C2B14D82A2B78D2182B89
:101FD00007D80A2B67D2082B00D0EAE03E21FF2069
:101FE0006BE0223B062B00D9E3E0D17808201E39B4
:101FF000C9B262E0352B6FD00DD8332B63D0342BB0
:1020000000D0D6E0794C04206179B943FEF71EFE7A
:102010006379BB4372E0362B72D0372B00D0C8E017
:1020200008260425714C042061793143FEF70EFE29
:102030006179A9435AE06D2B1BD8642B37D2492B09
:1020400071D0644A0CD8472B64D0482B00D0B0E044
:102050001168674B654C0B401360617920257CE06B
:102060004B2B73D062D34C2B00D0A2E003688022AC
:102070007AE0812B09D8782B00D380E01423D17823
:1020800002206D395943C9B217E0FF2B00D090E010
:102090000A991320FEF7DAFD6A4628215218534B9D
:1020A00012781A7585E0D1780020C9B205E00A23BC
:1020B0000920D17864395943C9B2FEF7C7FD78E0E9
:1020C000D17828395FE0494C042061793943FEF723
:1020D000BDFD63793B4311E004250826434C2800ED
:1020E00061792943FEF7B2FD6179B1432800FEF71B
:1020F000ADFD63791D4365716379B343637158E046
:1021000004253A4C28006179A94328E0374C08257A
:10211000617922E08021136849030B43334C13603B
:10212000617920250AE0036881221DE080211025C5
:10213000136849040B432D4C136061792943042033
:10214000FEF784FD63791D43657132E01025116847
:10215000284B264C0B40136061790420A943FEF7FD
:1021600075FD6379AB43C9E7520513430922036048
:10217000164B1A706A46194B928D1A8019E0282363
:10218000D17877395943C9B2032096E70320044038
:1021900024026418062C0CD1DB783E2B09D1694649
:1021A0000E4B898D198013681D4315600822074B5B
:1021B0001A70084A1368BB431360FFF73DF9C04625
:1021C00088130000DE020000B81E0100B0020020EB
:1021D000C04000506C05002076050020B2020020AF
:1021E000FFFFFFBF9407002001030020EB02002047
:1021F000FFFFEFFFFFFFFFFE07B5094A136A0093D9
:10220000084B196A019100991162019A1A62064BF2
:102210001B68002B02D000980199984707BDC04663
:102220000040005040400050DC0100201FB50E4926
:102230000E4A0B6A0C240193136A02930C4B186A22
:1022400003900298A04302900198086202991162DB
:10225000039A1A62074B5B68002B03D0019802991E
:10226000039A98471FBDC04680400050C0400050B0
:1022700000410050DC01002008B5044B08221A621E
:10228000034B9B68002B00D0984708BDC04000500E
:10229000DC0100200A4B800182B0C0180190019B34
:1022A000019A012012688840011C11431960054BF6
:1022B00020211A6800200A431A6002B07047C04605
:1022C000144000508041005010B50F2810D8094B21
:1022D0000F221C68104094432043012218601140D3
:1022E0000A0119681020814311431960002000E0A1
:1022F000014810BD804100500189FFFFF7B5294C0E
:10230000019400290AD10199019C01262568041C29
:102310001034A640341C2C430C6014E0012904D175
:10232000019C019D81402D680BE002290BD1019C8D
:102330000199061C0D6801210F1C1036B740814021
:10234000394329432160184901910121002A06D10E
:10235000019A019C814024688C43211C04E0019A6D
:10236000019C8140246821431160C0210F4C104A18
:102370008900022809D15058E3600E4B03408020A9
:10238000000403435350042308E05058A3600002A4
:102390008023000A1B0603435350082300201360C8
:1023A000FEBDC046DC400050D8400050DC0100209B
:1023B00000E100E0FFFF00FF30B5031E1D2B00D938
:1023C000CAE004F053FC0F1B22292B323232323286
:1023D00032323240464C52585F657382828282901C
:1023E00090A59EC05D4B002018605D4B18605D4B52
:1023F00018605D4B18605D4B1860AEE05A4B5C4A4C
:1024000019680A408021C901A2E0574B594A19684E
:102410000A40C02189019BE0514B00E04F4B1968F5
:10242000554A0A40F021090292E04D4A0121106804
:10243000DC1C0D1C053BA5409940A8430B1C011C4E
:102440001943116086E0484B4C4A19680A40042140
:102450007EE0454B4A4A19680A40082178E0424B21
:10246000484A19680A40102172E03F4B464A1968F1
:102470000A4020216CE03A4B444A19680A40802106
:10248000490065E0364B424A19680A4080211AE04B
:10249000354B404A19680A4003210A431A602F4B02
:1024A0003D4A19680A40C021090151E02C4B3A4AC3
:1024B00019680A40C02109010A431A60274B354AAE
:1024C00019680A40C021890042E0264A113B5B009E
:1024D0000321181C0D1C1468994008380B1C8540FA
:1024E0002343AB430BE0214A1168192B03D1294B3D
:1024F0000B40032102E0284B0B400C210B431360DF
:1025000028E0184BFF211A68120C12040A431A60C3
:10251000124BFF211A68120C12040A431A60124B64
:10252000174A19680A40802109010A431A6019688C
:102530001A4A0A40C0210A431A600C4B0D4A196816
:102540000A40302104E0094B144A19680A40C021AE
:102550000A431A60002000E0114830BD30000050EE
:1025600034000050380000503C0000504000005043
:10257000BFBFFFFFCFCFFFFF0F0FFFFFFBFBFFFF33
:10258000F7F7FFFFEFEFFFFFDFDFFFFFFEFEFFFFCD
:10259000FDFDFFFFFCFCFFFFF3F3FFFF3F3FFFFFED
:1025A0000189FFFFF8B52B4C012325681D4205D09A
:1025B0002360294B1B68002B00D0984702231D4243
:1025C00005D02360244B9B68002B00D09847042340
:1025D0001D4205D02360204B1B69002B00D098477B
:1025E00008231D4205D023601B4B9B69002B00D0A4
:1025F00098471A4D1A4C2F682668FB0608D52A689A
:10260000184B13402B60144B5B68002B00D098478D
:10261000FB0208D52A68144B13402B600E4BDB6875
:10262000002B00D09847F30608D522680D4B1340C5
:102630002360094B5B69002B00D09847F30208D553
:102640002268094B13402360034BDB69002B00D049
:102650009847F8BD44000440EC01002050000440BD
:10266000540004401F000F000F001F00F8B52B4C52
:10267000012325681D4205D02360294B1B6A002BCE
:1026800000D0984702231D4205D02360244B9B6A4B
:10269000002B00D0984704231D4205D02360204B17
:1026A0001B6B002B00D0984708231D4205D02360E8
:1026B0001B4B9B6B002B00D098471A4D1A4C2F6870
:1026C0002668FB0608D52A68184B13402B60144B6C
:1026D0005B6A002B00D09847FB0208D52A68144B90
:1026E00013402B600E4BDB6A002B00D09847F3069B
:1026F00008D522680D4B13402360094B5B6B002B00
:1027000000D09847F30208D52268094B1340236094
:10271000034BDB6B002B00D09847F8BD44001440FE
:10272000EC01002050001440540014401F000F0022
:102730000F001F00084BF022196812040A431A60A8
:10274000064BC022196892030A431A601968044AAA
:102750000A401A607047C046080200500C00005042
:10276000FFFFCFFF70B507260640321FD3B2012509
:10277000032B0AD91E4CF6002268B5400023AA4359
:10278000994200D02B1C13430BE01A4CD200236853
:1027900095402A1C1D1C00239543994200D0131C10
:1027A0002B432360C30622D5103807281FD804F016
:1027B0005DFA0406080A0C0E10160F4B0AE00E4BC9
:1027C0000EE00E4B06E00D4B0AE00D4B02E00C4B09
:1027D00006E00C4B19680C4A0A40082105E0094B39
:1027E00019680A4A0A40802109030A431A6070BD29
:1027F0000800044008001440500004405400044005
:10280000500014405400144007000F000F00070050
:10281000F0B5072385B003901840031C023B0C1C45
:102820000190B14A052B05D8181C04F01FFA0606C2
:1028300008080B0B5269920006E0526904E0D26965
:10284000920601E0D2691206920F05D0022A06D143
:10285000A64A1268029204E0A54E029601E0A54F36
:102860000297039E172E4CD8301C04F0FFF90C0C75
:102870000C0C121212124A4A4A4A4A4A4A4A232A5B
:102880002C2E30363B42039F9B48F90005680231ED
:1028900004E09A48039F0568F9001E3901228A4026
:1028A000E668111C95430022964200D00A1C2A4378
:1028B000026026E0924A93491068E7680140394374
:1028C0001EE08F4A0AE0904A0DE08F4A12E08F4ADC
:1028D0008C4910680140E06811E08C4AE168156895
:1028E00008040AE08A4A10688649E66801403143D4
:1028F00006E0874AE76815683804824929400143A1
:102900001160019E043EF2B200962678032A03D994
:102910007948019F056802E07848009F0568F90042
:10292000033101228A40111C95430022964200D0B7
:102930000A1C61682A430260002967D1E278052BEE
:1029400005D8181C04F092F9050507070C0C714B0B
:1029500002E0704B05E0704B1968FF20814304E0F2
:102960006D4B110218686D4A02400A431A60607884
:10297000A5686421684304F08DF9009E0138039036
:10298000F2B20723A678032A16D9654A0198176878
:10299000191C009787000098B94088433340BB401A
:1029A000011C019E19430C2373435E4F1160DA1919
:1029B000691E11605C4814E05C4A181C17683340BB
:1029C0000197009F009EB900019F88408B4087437C
:1029D0001F430C2373431760554F691EDA1955487E
:1029E000116003991B181960A3780126032B01D8E5
:1029F000514AD65CE1780298013104F04BF9311C60
:102A000004F048F9291C04F045F9FAE0029804F0B2
:102A100041F98023071C5B0500209F4200D9F0E0AC
:102A2000464B9F422FD9390C381C8EB204F032F934
:102A300080235B02984201D90136B6B280235B0045
:102A40009E4221D93E0A390E301CCDB204F022F943
:102A500080235B02984201D90135EDB200230122A7
:102A6000591C171CC9B29F40AF4201DC0B1CF6E792
:102A70004D1EAA40D5B20020102D00D9C1E037026A
:102A80008026760001E002260125311C381C04F066
:102A900001F9291C04F0FEF8071C80B2311C0090DB
:102AA000029804F0F7F8291C04F0F4F8009904F0F7
:102AB000F1F802900198013E0238052805D8FF235D
:102AC00004F0D4F809090B0B3E3E124AFF211368AB
:102AD0000E408B433AE00F4A33E00F4A1E40116824
:102AE00099430B1C32E0C04600020050F800002061
:102AF000001BB7000080510108000440080014408A
:102B0000500004400F000F005400044050001440D7
:102B1000540014400000044000001440FF00FFFF78
:102B2000040004400C000440100004400400144061
:102B30000C00144010001440B46F0000FFFF0100AF
:102B4000314A1E403302314916680E401E43681E4A
:102B500016600F2812D804F089F8080A110C111118
:102B6000110E1111111111111110042506E000258B
:102B700004E0012502E0022500E00325039E6078C1
:102B8000F60607D5A36864215F1E5843BFB204F060
:102B900081F806E0009E013F70436421BFB204F05B
:102BA00003F9019A0138043AD1B280B2072303290C
:102BB00015D9174A019E1468B1001D402E1C8B4088
:102BC000251C8E409D433543019E0C2373431149C0
:102BD00015605A181760104A9B18186010E00F49CA
:102BE00094000E681D40A3409E430C235A43A54009
:102BF00035430B4E0D6093191F600A4FD2191060B8
:102C0000029805B0F0BDC04600001440FF00FFFF71
:102C1000040004400C000440100004400400144070
:102C20000C0014401000144010220423002921D06D
:102C300010420FD0184203D0204B14389A6F03E093
:102C40001F4B07219A6F084001218140081C104347
:102C5000986731E00122184205D01A4B04381968F0
:102C600082400A4327E0184B82401968101C084331
:102C7000186021E010420ED0184203D00F4B1438D8
:102C80009A6F03E00E4B07219A6F084001218140A3
:102C90008A439A6710E00122184206D0094B043893
:102CA0001968824091430A1C05E0074B824019686D
:102CB000101C0A1C82431A607047C0460000144072
:102CC000000004407C0014407C00044007231840AE
:102CD0000322023800B5104B1140052804D803F038
:102CE000C5FF08080F0F131358690C4A0907024063
:102CF00003E05A698907920092080A435A6109E081
:102D00000901DA69302002E0DA698901C0208243D2
:102D10000A43DA6100BDC04600020050FFFFFFCF4A
:102D2000034B002058605B68DA0700D50148704704
:102D3000FC0000500296FFFFA023DB059A680121EA
:102D40000A439A607047000008B5A023DB059A6922
:102D500010210A439A61034B1B68002B00D098474F
:102D600008BDC0462C02002010B50123232805D140
:102D70000D4A1940C9005368082006E0222808D1EE
:102D8000094A194053688900042083430B43536068
:102D900008E0064A83401468002901D01C4300E083
:102DA0009C43146010BDC046000200500802005051
:102DB00008B5054B40211A680A431A60034B5B684B
:102DC000002B00D0984708BD000200502C020020C4
:102DD00000487047001BB70030B5154B85B06A46F8
:102DE00023CB23C21B686C461360124B1A6A191C52
:102DF000100301D5104A00E0104A096A0D4BCD03BB
:102E000012D4186A196A1D6AC005C00D89042D0400
:102E1000C90EAD0F023050430231AD0003F03AFF4E
:102E2000615903F037FF00E0002005B030BDC04617
:102E3000B86F00000002005000805101001BB70075
:102E400010B50E4C072322691A420CD022691A4091
:102E5000022A02D1FFF7C0FF08E022691340032BCA
:102E600003D1074802E0074800E00748A1690F23A3
:102E70001940013103F00EFF10BDC04600020050A2
:102E800010270000001BB70000805101F7B5042196
:102E90008020D64BD64ADC6811621968C004014311
:102EA000802019601968C005014319600021D14BC9
:102EB000D1481980036800929B063AD4CF4B1D7805
:102EC0001900092D35D8CE4D2E68B2000FD4CD4E45
:102ED0003678002E0BD029684A052AD429684A0280
:102EE00027D419780131C9B219701B7809E0C64B93
:102EF0001B78DBB2002B17D00B780133DBB20B70E1
:102F00000B780A2B15D180250521C04B1D70C04BB5
:102F10001970C0498B682B438B604021009B009A3D
:102F20009B688B43936004E00725B9490D70B7494E
:102F30000B700021B84B1980C82C00D8C7E10225BE
:102F4000AF490E680B002E4200D195E10E680E3598
:102F50002E4202D00B68AB4314E00E68AF4DB206B0
:102F600000D424E104260F6837420DD140200B68BD
:102F70001E430E600A6882430A60AC4200D9A6E193
:102F80000B6803430B60A2E180270968B143196015
:102F90001E68BE431E60AC4202D8196839431960EE
:102FA000402619681C68490831403440A14200D0CD
:102FB0008DE11C689A49220600D4E4E00C78012CCB
:102FC00000D87BE10125974C64792C423CD0964C8B
:102FD0002568002D38D1954C276ABC466246944F2F
:102FE000174004222762934FFA67276A033A9743F0
:102FF00080222762904FD2053C68144308223C602F
:103000008E4C8F4F2570BC681443BC60009A946846
:103010002643966080260468760234430460894C17
:103020002570894C2578FF2D0FD165780324A543A1
:10303000FC2D0AD1854DAC683443AC608025046812
:103040006D012C43046000E00878814E0C783578DF
:103050007D48E4B2EDB205550024250001960E78B6
:10306000B44204D8065D01347540E4B2F7E7002DA0
:1030700000D023E13F260478B443802C5FD1196847
:10308000CA000CD50178734CC9B221704178724CDA
:10309000C9B2217080241968A400214319606149D4
:1030A0004C79E2060FD5CD7A0478A5420BD10D7B81
:1030B0004478A54207D180251C686D042C43002567
:1030C0001C60664C25804C79A20600D4F6E04D7B4E
:1030D0000478A54200D0F1E001248D7B4178A14322
:1030E000A94200D0EAE04178484E2140484D0BD03B
:1030F0000021424A1170802232701968584A0A40F1
:103100001A6005222A70D9E00222564887681743C0
:10311000876087689218974387603E4F7C32B86813
:103120009043B8604027009A9068384390603170AF
:1031300081211A6889050A431A602C70BEE01A685A
:10314000494C4A4E22431A602A00494C257000948B
:103150000C783700A446541CE4B2944505D9855C2C
:10316000EDB2B55401252200F2E7002D01D0009800
:10317000027001980A780078D2B2C0B2B854F22036
:103180001A6882431A6032480A7800782E4CD2B20C
:10319000C0B2A05420201A6882431A600A78013213
:1031A000D2B20A700A78102A00D987E08FE0284945
:1031B0000A785200D2B20A70AC4203D80A780132BF
:1031C000D2B20A702B490A780132D2B20A700A7858
:1031D000072A05D920201A6802431A6000220A70C3
:1031E00010211A680A431A6071E0C046200011409D
:1031F000C0400050700500208007002072050020AC
:103200006C050020160300206605002076050020CE
:10321000B00200200040005074050020FF050000AF
:103220003E040020EB020020E002002000000E40DF
:10323000FFF7FFFF04E100E000001140BC020020A6
:10324000804000503F050020C002002000020050D6
:1032500017030020270300207C070020860700209A
:10326000FFFFBFDF00410050010008000103002004
:1032700034020020790700201549164A8C4219D9DA
:10328000117812291AD91968490702D519682943F2
:10329000196004201968014319601968890716D557
:1032A0001968FB30814319601968F53801431960CA
:1032B000002309E013780133DBB207E01968064AFE
:1032C0000A401A600023034A1370044A1370F7BDC2
:1032D000FF0500007907002000FFFEFF3E040020EC
:1032E00008222F4B2F49F0B51A620A682E4B134063
:1032F0002E4A0B6013685B0350D580241068A4022B
:103300002B4B204206D110682043106080201C788F
:10331000204306E014682748204010607F201C7876
:1033200020401870802005250B68C00403430B6003
:10333000214B224F1C78E4B2601CC0B218702048A8
:1033400005551C78E4B2651CEDB21D7004250555C9
:103350001C78E4B2651CEDB21D70002505551C7883
:10336000E4B2651CEDB21D703D78EDB26E1CF6B294
:103370003E7005551C78E4B2651CEDB21D708725C2
:1033800005551C78E4B2651CEDB21D7013689B03F3
:10339000DB0F03550A680B4B13400B60F0BDC046B2
:1033A000C04000506C050020FFFFDFFF80070020B9
:1033B000B0020020FFFFFDFFEA02002040050020D0
:1033C0003F040020FFFFFFFBF7B5C84AC84C138835
:1033D000019401339BB21380C64A138801339BB218
:1033E00013802388002B03D02388013B9BB22380CA
:1033F000C14A13780133DBB21370C04B1A68002A3C
:1034000002D01A68013A1A60BD4A1388002B06D10F
:10341000BC4BBD481A68BD4ED2010FD441E01388A1
:10342000013B9BB2138013889BB2002BF0D1190093
:10343000B74AD15401330A2BFBD1E9E7B54AB64963
:103440001278802A03D10A88013292B200E0002269
:103450000A800988B14A914223D98025B049812741
:103460008A689024AA438A60AE49403D8A68BF05B5
:103470002A438A600021AC4A3C3D1570A54A117070
:103480001A683A431A600768A84A3A40A84F02608F
:10349000BA682243BA608027A64ABF01D767D567BA
:1034A0003170A5490A88002A0BD00A8892B2551EAD
:1034B000ADB20D80012A04D120259D498A68AA4316
:1034C0008A609E490A88013292B20A809C490A8821
:1034D000002A03D00A88013A92B20A80994D9A4A8A
:1034E000298800290CD02988013989B22980974977
:1034F00011802988002903D140250168A943016072
:103500001188002909D01188013989B211801288E7
:1035100092B2002A01D18E490A708E490A78D2B23D
:10352000002A0ED0FA278C4DBF006A88BA4202D812
:1035300001326A8014E000226A800A78013AD2B22D
:103540000DE08649097800290AD07249097849B204
:10355000002905DB1D6882492940196081490A70EC
:10356000814A118889B24D1CADB21580C8291DD180
:1035700080276B4DA968B943A9606A4D403FA9688F
:103580003943A9600021774D3A3F2970774D298052
:103590001D687749294019605E49634D0F70317885
:1035A000C9B2002901D1297000E02F701288C72A02
:1035B00021D81A6852041ED500214027694A584D67
:1035C0001170AA6880310A43AA60564DAA68BA43AE
:1035D000AA60504A1170544A7B3911701968654AC3
:1035E0000A4080211A600268C9040A43026019680F
:1035F000614A0A401A60614A116800290AD01168BC
:10360000013911601268002A04D1102545498A68E1
:10361000AA438A605A498A79002A0FD04E4A97886D
:103620007D1C95800A258C796543AF4206D18027A1
:103630001D683F043D431D6000259580514A158853
:103640000135ADB215803578EDB2002D00D1ADE079
:103650004D4D296801312960C8212F6889008F42AA
:1036600000D8C4E000212960484D2F680F253D4057
:10367000474F40353D709027464D31702970464D7B
:103680002B4E2970B5683D43B5600126334D103F80
:103690002E70234EB568BD43B560224E403FB568DD
:1036A0003D43B560204D019C2970304D29801E6836
:1036B0002F4D354004261D60384D2E60FA25AD0093
:1036C00025800625134C2570264C21701D68294C39
:1036D00025401D60324C02252170324C2170324948
:1036E0008C6834438C608C6878E0C04628030020E6
:1036F000E40200207A0700204D050020E0020020AF
:103700003A0300206C050020800700209407002069
:10371000180300207605002086070020B036000040
:1037200000400050C0400050B0020020FFFFFBFFEF
:103730008040005004E100E0BE020020420500206D
:1037400092070020A4020020240300208813000018
:103750004C0500206A0500203402002016030020DA
:10376000FFFFBFFF7205002074050020B202002099
:10377000FFFFFFBFFFFFBFDFFFBFFFFF48050020C8
:10378000EB020020680500208C070020B802002012
:103790003D040020780700209507002000E100E0AC
:1037A000EA020020880700200000154049794907F7
:1037B0001DD5874C218889B24E1CB6B22680FA26C8
:1037C000B600B14213D92580102582490C692C42DC
:1037D00006D08C68AC438C608C6870352C4305E057
:1037E0008C682C4380258C608C68AC438C60802175
:1037F00000688902084035D01388DBB2802B00D0E6
:10380000E5E0754A754B9179012916D000290AD057
:1038100002291ED198680143042099609968814368
:103820009960032313E00420996801439960996823
:10383000023881439960012309E002200424996839
:10384000014399609968214399609071BFE0937139
:10385000BDE0002191719A6802318A439A609A68AA
:103860000231B2E05E495F4C0D88002D13D00D8807
:10387000012D0CD11E685C4D35401D605B4B1B78E3
:103880005BB2002B02DA0523237000E020700B8866
:10389000013B9BB20B802078C0B2092800D996E08A
:1038A00003F0E4F905132A303D5C61777B82FA224C
:1038B0004F4B92001988914200D088E000220421E9
:1038C0001A80464A93684B403FE013888022DB050C
:1038D000DB0D5200934200D079E03F4BD879421C77
:1038E000DA71052873D803F0C1F903320332723656
:1038F0003A4A0421936827E012880221374B920646
:103900000BD504E012880221344B120605D59A68C3
:103910000A439A609A68491857E09A6855E01388F4
:103920008022DB05DB0D5200934250D12A4BD8791F
:10393000421CDA7105284AD803F098F903090309F3
:10394000490D0221254A93680B4393603FE0234BC6
:1039500004219A6835E00022DA7138E004211F4B17
:103960009A680A432EE0FA22214B9200198891426C
:103970002DD100221A80184B1A7A511C1972042179
:10398000164BD2071CD49A680A439A609A6802219F
:1039900014E0124B04219A680CE0128804210F4BAA
:1039A00052060DD59A6809E0128804210B4B520685
:1039B00006D59A680A439A609A6802390A4305E074
:1039C0009A688A4302219A609A688A439A60F7BD8E
:1039D000700500208040005034020020004100505B
:1039E000B2020020B0020020FFFFFFBF76050020DA
:1039F000740500208021E34AF0B5136849020B43A7
:103A0000E1491360087885B0C0B2431CDBB20B708B
:103A1000042801D900F0A8FD8023DB0503F026F976
:103A2000080E080328000820D8498A6882438A6063
:103A3000D7490A6813430B6000F096FDD44801682B
:103A40000B4303600820D1498B6883438B60136864
:103A50005B0305D58021CF4A490293680B439360ED
:103A60000221CD4B9A680A439A601B6800F07CFDE6
:103A70008020CA49C0040B78013BDBB20B70C84BF5
:103A800019680143802019601968C0050143196055
:103A9000C449D8688842FCD900210124C24B0426BD
:103AA0001970C24B1970C24B186A2043B94C186286
:103AB000A568C04828404025A060BF4CA068A84326
:103AC000A060BE4806608026186A3601304318623E
:103AD000BB48437901902B4201D100F0B3FCB94BB4
:103AE0001E781D008E4201D100F0ACFC1E780F2E16
:103AF00001D800F0A7FC1E78EF2E01D900F0A2FC3F
:103B00001B78B14E0F3BDBB2F35CDBB2402B25D10F
:103B10001368DB0401D400F095FC13685B0301D447
:103B200000F090FC80220A25A848D20403681343C1
:103B30000360A74B1C78E4B2621CD2B21A70A54A8B
:103B400015551C78E4B2651CEDB21D70092515559C
:103B50001C78E4B2651CEDB21D703CE29908C8B255
:103B6000072847D003D8002807D000F06BFC0E3997
:103B7000012900D8B1E100F065FC69780E2901D86F
:103B800000F060FC1020A1688143A16069780F39C2
:103B9000715CC9B20291402901D100F053FC8E49F9
:103BA000087840B2002804DA3F200C7804400194E1
:103BB0000AE08878C0B2C8704878C0B288700878C7
:103BC000C0B24870002001900F248878A0430024E0
:103BD000E02801D08C70CC700020804C275C0E5CFB
:103BE0002500B74201D000F044FC01300528F5D192
:103BF00000F049FC69780E2901D800F023FC102759
:103C0000A168B943A160A9780F2907D9E978EF29FC
:103C100004D8AB780F3BDBB2F35CDBB2012B06D0F0
:103C2000002B06D0072B00D197E000F00BFC80237F
:103C30005B0029780F39C9B2775C6978FFB20F3918
:103C4000C9B2755C6449EDB20C7864B2002C01DA3B
:103C50000C7808E08C78E4B2CC704C78E4B28C70CC
:103C60000C78E4B24C7000200E78029076B2864256
:103C700003DA0C783F210C4002941268520300D4FE
:103C8000E0E3BA01AA18564DD2B2698952189B18BE
:103C90009BB25B08019A6B81527952B2002A00DB19
:103CA000D0E3019A4F490D88D07C0A2242439542C5
:103CB00000DCC7E300260E80802108274348C904A2
:103CC00002680A430260424A1578EDB2691CC9B223
:103CD000117040494F551578EDB26F1CFFB2177047
:103CE00007274F551578EDB26F1CFFB217704E5570
:103CF0001578EDB26E1CF6B216703B4EB4466446B3
:103D00003678F6B2771CFFB227704E5515786C46A0
:103D1000EDB26E1CF6B21670A6264E551578247AB2
:103D2000EDB26E1CF6B216702B4E7678F6B24E558A
:103D30001578EDB26E1CF6B216704C551478E4B2DC
:103D4000651CEDB21570DDB20D5514781B0AE4B296
:103D5000651CEDB215700B5576E12B780F3BDBB28D
:103D6000F15CCBB202936B780F3BDBB2F35CDBB25E
:103D70000393194B1C7864B2002C37DA1C783F236C
:103D80001C403DE080070020BC0200208040005025
:103D900000001140000200500000054026030020F2
:103DA0002000114061020000790700203E0400203D
:103DB00000000E40FFFFFEFFC040005000E100E0A9
:103DC000EB020020A6020020000000206C0500206D
:103DD000EA0200203F040020C00200201803002057
:103DE0003402002028030020400500209C78E4B223
:103DF000DC705C78E4B29C701C78E4B25C700024E7
:103E0000019B9B7C002B00D11CE3019BED4D2E8878
:103E1000987C642343439E4200DC13E300262E80FB
:103E200013685B0300D40DE380220927E648D2041F
:103E3000036813430360E54B1D78EDB26A1CD2B2F0
:103E40001A70E34A57551D78EDB26F1CFFB21F7010
:103E5000082757551D78EDB26F1CFFB21F705655DD
:103E60001D78EDB26E1CF6B21E70DA4EB446614695
:103E70003678F6B2771CFFB20F7056551D78EDB24A
:103E80006E1CF6B21E70AA2656551D78EDB26E1C39
:103E9000F6B21E70FF2656551D78EDB26E1CF6B2B6
:103EA0001E70CD4E7678F6B256551D78EDB26E1C6A
:103EB000F6B21E7054551C78E4B2651CEDB21D704C
:103EC000012515551C78E4B26519EDB21D70029BF1
:103ED0009901039B5918C9B2B5E01168C90400D40F
:103EE000B0E21020A1689B018143A160DCB26B7835
:103EF000B9490F3BF35C4878DBB2FB38042800D9A2
:103F0000A0E202F0BDFEFB0105000500A600A60030
:103F10008021C902402B3ED012680A4200D191E2B2
:103F200080210A26A84AC90412680A43A6490A60E1
:103F3000A64A1078C0B2411CC9B21170A4490E54EF
:103F40001078C0B2461CF6B2167009260E541078CE
:103F5000C0B2461CF6B2167000260E541078C0B2DD
:103F6000461CF6B216709B4EB44665463678F6B2DD
:103F7000771CFFB22F700E541078C0B2461CF6B2F8
:103F80001670B3260E541078C0B2461CF6B21670E6
:103F9000FF260E54C9E013680B4200D152E2802282
:103FA0000A248948D204036813430360874B1978B5
:103FB000C9B24A1CD2B21A70854A54541978C9B28F
:103FC0004C1CE4B21C70092454541C78E4B2611CEB
:103FD000C9B21970002111551D787E4FEDB26C1CCD
:103FE000E4B21C703C78E4B2661CF6B23E705455E4
:103FF0001C78E4B2651CEDB21D70B32515551C7814
:10400000E4B2651CEDB21D70FF2515551C78E4B2B5
:10401000651CEDB21D7011551C78E4B2651CEDB243
:104020001D7011551C78E4B2651CEDB21D70115560
:104030001C78E4B2651CEDB21D7011551C78E4B219
:10404000651CEDB21D7011550268644B134003608E
:10405000F8E18020C002402B00D1C5E01268024286
:1040600000D1EFE180210F26574AC90412680A43A4
:1040700055490A60554A1078C0B2411CC9B2117046
:1040800053490E541078C0B2461CF6B2167004267E
:104090000E541078C0B2461CF6B2167000260E54AC
:1040A0001078C0B2461CF6B216704A4EB446654649
:1040B0003678F6B2771CFFB22F700E541078C0B26B
:1040C000461CF6B21670B4260E541078C0B2461CC8
:1040D000F6B21670FF260E541678F6B2701CC0B2F7
:1040E00010703D488778FFB28F551678F6B2771C6E
:1040F000FFB21770C778FFB28F551678F6B2771CEB
:10410000FFB217700779FFB28F551678F6B2771C99
:10411000FFB217704779FFB28F551678F6B2771C49
:10412000FFB217708079C0B2885510782343C0B2AF
:10413000461CF6B216702A4E0B54B378294C0F3B2E
:10414000E35CF0789B010F38205CDBB2034310780E
:10415000C0B2471CFFB217700B5433790F3BE05CC1
:10416000737980000F3BE35CC0B2DBB21F093843B8
:104170000090684617781B01FFB27D1C0571057918
:1041800000981570C855B079DBB20F38205CC0B20A
:1041900087083B4300936B4617788001FFB27D1C74
:1041A0001D711D79009B1570CB55F3790F3BE35CB6
:1041B00018431378C0B2DBB25C1CE4B21470C8546C
:1041C0003AE1C0467A0700206C050020EA02002090
:1041D0003F04002040050020C0020020FFFFFFFB3D
:1041E000A6020020000000201368034200D129E14C
:1041F00080220F25DD4CD204236813432360DC4B5F
:104200001878C0B2421CD2B21A70DA4A1554187823
:10421000C0B2451CEDB21D70042515541D78EDB2D9
:10422000681CC0B21870002050551D78EDB26E1C8D
:10423000F6B21E70D04E0195B44665463678F6B299
:10424000771CFFB22F70019D56551D78EDB26E1C84
:10425000F6B21E70B42656551D78EDB26E1CF6B23D
:104260001E70FF2656551D78EDB26E1CF6B21E70FC
:104270008E78F6B256551D78EDB26E1CF6B21E70F1
:10428000CE78F6B256551D78EDB26E1CF6B21E70A1
:104290000E79F6B256551D78EDB26E1CF6B21E7050
:1042A0004E79F6B256551D78EDB26E1CF6B21E7000
:1042B0008979C9B251551978C9B24D1CEDB21D703A
:1042C00050541978C9B24D1CEDB21D705054197874
:1042D000C9B24D1CEDB21D7050541978C9B24D1CB5
:1042E000EDB21D7050541978C9B24D1CEDB21D705D
:1042F00050542268A14B13402360A3E0402B00D10F
:10430000A0E01268520300D49CE080210A26974A5C
:10431000C904126823430A4394490A60944A1578F1
:10432000EDB2691CC9B2117092494E551578EDB2C3
:104330006E1CF6B2167009264E551578EDB26E1C3D
:10434000F6B2167000264E551578EDB26E1CF6B218
:104350001670894EB44660463678F6B2771CFFB2C6
:1043600007704E551578EDB26E1CF6B21670B52674
:104370004E551578EDB26E1CF6B21670FF264E55EE
:104380001578EDB26E1CF6B216707D4E4B55B378B3
:104390007C4D0F3BEB5CF4789B010F3C2C5DDBB25A
:1043A00023431478E4B2671CFFB217700B553379BE
:1043B0000F3BEC5C7379A4000F3BEB5CE4B2DBB227
:1043C0001F093C4300946C4617781B01FFB2781C10
:1043D00020712079DBB210700098C855B4790F3C79
:1043E0002C5DE4B2A7083B4300936B461778A40109
:1043F000FFB2781C18711879009B1070CB55F379B7
:104400000F3BEB5C1C431378E4B2DBB25D1CEDB2F6
:104410001570CC5413785C4DDBB25C1CE4B21470A4
:10442000EC79E4B2CC541478E4B2631CDBB21370C0
:10443000C0232A7A13430B554C4B1A684F4B134039
:104440004A4A13601021514B1A680A4205D00320D2
:104450004F4A10601A688A431A6019684D4A0A4028
:104460001A6000231900464AD1540133082BFBD1AE
:104470007AE00023484A1373CA5CD2B2EA5401338B
:10448000052BF9D1DEE7444C207B451C2573012820
:10449000D8D11268520362D580200926334CC0045B
:1044A00022689B0102432260314ADBB21578EDB2EB
:1044B000681CC0B210702F4846551578EDB26E1CBE
:1044C000F6B21670082646551578EDB26E1CF6B297
:1044D0001670002646551578EDB26E1CF6B21670B1
:1044E000254E0395B44665463678F6B2771CFFB282
:1044F0002F70039D46551578EDB26E1CF6B21670FE
:10450000A52646551578EDB26E1CF6B216704E789B
:10451000F6B246551578EDB26E1CF6B216706E46C0
:10452000367946551578EDB26E1CF6B21670CE7817
:10453000F6B246551578EDB26E1CF6B216708E784E
:104540000321314041551178C9B24D1CEDB21570AF
:10455000029A134343542268084B13402360C82235
:104560000E4B92001A806DE705B0F0BD6C0500207F
:10457000EA0200203F04002040050020FFFFFFFB6F
:10458000A602002000000020C002002080070020BA
:1045900048050020FFEFFFFF340200203A0300200F
:1045A000F7B56A46234BD01D1B680127DBB20370A9
:1045B00000231D001E001C0001781F4AC9B2517360
:1045C0009373D373082B09D0394202D001260134EA
:1045D000E4B201334908DBB20125F3E7002E00D035
:1045E0009473002D02D008235173D373937B042B53
:1045F0001FD1124B1A68520307D51024104A916834
:10460000214391601A6822431A600E490B78DBB28D
:104610005A1CD2B20A7002780B48D2B2C2540B783C
:10462000092B06D90023094A0B709168084B0B40EF
:104630009360F7BD00000540340200208007002091
:10464000C04000503F050020A6020020000200509C
:10465000FFFFFEFFF0B5BD4C87B0236804AADBB2B4
:10466000D11D0B70A3691B07DD0F002B00DB51E18F
:10467000082640277F22A3693343A36108780B787B
:1046800038401340002800D1BCE07D2B00D1B5E0BC
:104690007E2B00D0BAE2AE4D2B78002B00D08DE0FF
:1046A0008021AC4A93688B439360AB4A93681F4365
:1046B000AA4B97601B78DBB2002B06D08021A84A5A
:1046C000C90113680B43136004E00621A54A117069
:1046D000A54A1370A54A1378DBB2002B03D01378D8
:1046E000013BDBB268E00B22A14DA2492A70013ADE
:1046F0006A70E632AB70EB702A71EE3A6A713C3246
:10470000AB71EA710A68120E2A720A68120CD2B2F0
:104710006A720A68120AD2B2AA720A680C21D2B26C
:10472000EA72954A1170954A1370954A13748C4A2F
:10473000944B11680B4013601022E3681343E3604D
:10474000E36892181343E360E368183A1343E360A5
:10475000A369DB00FCD52E787C4BF6B21E603000DE
:1047600000F01CFB0127B74215D8A3691B02FCD43B
:10477000824A7649137801370133DBB21370EB5C60
:10478000FFB2DBB20B601378DBB2EB5C5840C0B217
:1047900000F004FBE7E7A3691B02DB0FFBD16B4AC8
:1047A000764910600A780132D2B20A70764A1370E4
:1047B000764A1360664A0233137046E22B78022B66
:1047C00000D042E200F0DCFA0021684B6F4A18701A
:1047D0006F482970116011684C1C14608142FAD92D
:1047E000002111601A788A4200D02EE2614A1268D4
:1047F000D2B21A700F2219780A405BE00022634B94
:104800001A6022E2002B17D180245F4864000278EE
:10481000D2B2511CC9B201705E49520054520278A2
:104820005200535280210378554ADBB213745A4A1E
:10483000090613680B4366E0454B1B78DBB2022B7D
:1048400063D0032B00D0E1E1544B09781A781F2381
:104850000B40934200D0F8E110214C4A1060E3680D
:104860000B43E360E36849180B43E360E3683343B9
:10487000E3600292A3693549DB00FBD5384B1A6827
:104880008023DB041A4002D001230B60DDE13B4BA7
:1048900039481F7805781E00AF4201D10A60D4E183
:1048A0001A78334DD2B2AD5CEDB22A1F3B2A03D940
:1048B0000278D2B21A70C8E10D60280000F06EFADA
:1048C0000127A3691B02FCD43378294A0133DBB2E8
:1048D0003370D35C1D49DBB20B6033780137DBB238
:1048E000D35CFFB25840C0B200F058FABD42E8D2E3
:1048F000A3691B02DB0FFBD1144A1060327801322E
:10490000D2B23270029A13609FE11D4B1D741F4B8F
:1049100018607BE1204A1C4D10681E4B002800DB0C
:104920005FE1174E307C40001F5AC0203840029093
:1049300036D011684900490811600021327C013AE3
:10494000D2B22A702A78520099527EE100001540B6
:104950009407002000400050C04000501603002083
:104960006C050020B0020020760500203D040020E8
:104970003F040020B8020020EA0200209007002037
:1049800034020020FFFFFFFB880700208C07002077
:10499000FFFF0F0078050020800700203C04002066
:1049A0002F78F8B2019002AF0130F871F8792870D1
:1049B000019809784700D953317C4900595A002998
:1049C00000D123E1317C49005F5A317C2E780231DD
:1049D000C919C9B2B14200D018E1297802A8C9B2F8
:1049E0004E1CF6B22E7080264900B6005E52297821
:1049F0000088490058520298136806005B005B0863
:104A00001360934F934A3B7C39005B009B5A013300
:104A1000B3420FDB3B7CF318DBB25B009B5A8E4A40
:104A2000DBB29355935D01365840C0B200F0B6F941
:104A3000F6B2E6E7894A1378DBB2022B05D0032BE6
:104A400000D0E3E00022864BC9E0834B002804D06D
:104A500000231370FF22834B2CE71A791E00702A63
:104A60007ED100217E4F804E3960587A3268120E16
:104A7000904200D0CAE09A7AFF2094463268120C25
:104A80000240944500D0C1E0DA7A94463268120AB6
:104A90000240944500D0B9E01A7B36680640B24225
:104AA00000D0B3E003226D4E32705B796F4ADBB207
:104AB00013701378DBB28B4203D13370694B1870DB
:104AC000C3E039602B786A4ADBB21370694B6A4ADB
:104AD000186802401A60694A69485579AD0718D5C7
:104AE0008027684E0170B568BD43B560664E403F93
:104AF000B5683D43B560654D297065490D78052D54
:104B000001D1023500E006250D70002561490D70C8
:104B100001E001210170102551799026A9435171BE
:104B200052790C3D5C492A4216D08A68B2438A60A9
:104B30000278002A6AD00021584A11801868584A21
:104B400002401A60574A1560524A1170564A117055
:104B50001968564A0A4042E08B6833438B6055E03F
:104B60001A79722A1FD100253D4A3F481560597AAB
:104B70000268120E914249D1FF219E7A0268120CFE
:104B80000A40964242D1DE7A0268120A0A409642F0
:104B90003CD11A7B03680B409A4237D12F4B1D70D2
:104BA000304B197051E018781F785A78C0B2013232
:104BB00097422BDD5A780132D2B20A740F7C1A78F0
:104BC000D21BD2B21A7000220132D7B2B84200D83A
:104BD00043E70F7CBF18F75DFFB2B754F4E71A60E4
:104BE00014E02878013840001E5A80204000864298
:104BF0000CD12878C0B2461CF6B22E70097840005D
:104C000019528021136809060B431360A369284ACF
:104C10001B0403D5022193680B439360A269244BC4
:104C2000D20707D501219A690A439A619A684918FF
:104C30000A439A60A3699B0603D41D4B9B69DB065C
:104C400003D50222A3681343A36007B0F0BDC0469A
:104C500034020020780500203C0300209407002047
:104C60008C0700203D040020B80200203C040020F6
:104C7000950700206C050020FFFFFBFFEB020020E2
:104C80001603002000400050C04000506605002080
:104C9000B00200207605002080400050B2020020C3
:104CA000FFFFFFBF00E100E072050020FFFFBFDF54
:104CB0000000154010B5FBF7BBFFFEF73DF810BD37
:104CC00070B51B4C072322691A4E1340052B02D8DE
:104CD000022B04D000E004239B00F0581AE0256A60
:104CE00001232D04AD0FAB4292415242AD1A226A0C
:104CF000D20C1A4201D0104B00E0104B206A216AFE
:104D0000C005C00D8904C90E02305843023101F0BC
:104D1000C1FFE840A1690F231940013101F0BAFF3A
:104D2000074B70610749C01801F0B4FFB06170BD56
:104D300000020050E400002000805101001BB70079
:104D400020A1070040420F00704700000B4B1A786B
:104D500019785200D2B24A4052001978D2B24A4071
:104D600012011978D2B24A401978D2094900521872
:104D7000D2B21A701878C0B27047C04644050020FD
:104D800010B5FFF7E3FF0F23034A18401378C0184C
:104D90001F231840107010BDB40200200023C2076A
:104DA00000D55E33820701D5BC225340420701D5AE
:104DB00061225340020701D5C2225340C20601D5E9
:104DC0009D225340820601D523225340420601D53D
:104DD0004622534040B2002801DA8C22534018008A
:104DE00070470000F0B5D24BD24C1A78237893B0BC
:104DF0009A4201D101F064FE80232278CE4D5B00FF
:104E0000002A12D1FF32FF32AA5A19009A4202D167
:104E10008022520015E02378DBB25A1CD2B22270F5
:104E20005B00EB5A8B42F6D1F2E72278013A52004E
:104E3000AA5A9A42ECD02278D2B2511CC9B221703F
:104E4000F5E723785B00EB5A934204D123780133D2
:104E5000DBB22370F5E723785B00EB5A002B01D11E
:104E600001F02EFE23785B00EB5A0233DBB2019394
:104E7000019A2378D318DBB25B00EA5A80239B00A7
:104E80009A4201D001F01CFE002630002378019ADE
:104E9000D318DBB25B00EE52019AF3B29A420FD9FB
:104EA0002278D2B2531CDBB223705200AA5AD3B27A
:104EB00002AA93554340D8B2FFF770FF0136EBE7E3
:104EC000802223789D490133DBB223700B68D20422
:104ED00013430B60002845D0994B02AA1B789278A7
:104EE0009A423FD100200625964B974F18701C78A8
:104EF000E4B2621CD2B21A70944A15551C78E4B21E
:104F0000651CEDB21D70052515551C78E4B2651CB5
:104F1000EDB21D7010551C78E4B2651CEDB21D7029
:104F20003D78EDB26E1CF6B23E7015551C78E4B2B9
:104F3000651CEDB21D70862515551C78E4B2651C04
:104F4000EDB21D70022515551C78E4B2651CEDB25A
:104F50001D7002AB1B791355754B18707C4B186094
:104F600001F0D7F9012702AB9D78754B1A781C0028
:104F7000954211D1774A02A9107809790130884207
:104F800009D01078744EC0B23070002903D0734E2F
:104F900030683843306011701B789D4201D001F0B9
:104FA0000AFC8021654AC90413680B43136002ABF5
:104FB0005B791100102B01D100F081FD00D999E03F
:104FC000072B00D1FEE14DD8032B00D155E13FD88E
:104FD000012B00D10EE1022B01D001F0ECFB0620E9
:104FE0000526584B1978C9B24A1CD2B21A70574AD2
:104FF00050541978C9B2481CC0B218705654197868
:10500000C9B2481CC0B21870002050541978C9B2F7
:10501000481CC0B218704C48844665460078C0B23F
:10502000441CE4B22C7050541978C9B2481CC0B268
:105030001870832050541978C9B2481CC0B2187037
:1050400056541978C9B2481CC0B218700023EAE15E
:10505000052B00D157E100D906E3404A404B1168C7
:105060000B404DE10B2B00D1B9E308D8092B01D13E
:1050700001F061FB334A354900D82EE3DAE30E2B09
:1050800000D174E301D901F015FB0C2B01D001F024
:1050900092FB05202B4B2C4D1978C9B24A1CD2B279
:1050A0001A702A4A50541978C9B2481CC0B21870F4
:1050B000042050541978C9B2481CC0B2187000209E
:1050C00050541978C9B2481CC0B218702878C0B2C0
:1050D000441CE4B22C7050541978C9B2481CC0B2B8
:1050E00018708B2050541978C9B2481CC0B218707F
:1050F000FF2398E1172B01D101F09CF932D8132B33
:1051000001D100F084FF09D8112B01D100F08FFDEF
:10511000122B01D100F03EFD01F04DFB152B01D10A
:1051200001F03DFA01D801F06FFA01F0E4F8C04651
:105130008807002095070020780500206C050020D6
:105140003C040020EA020020400500203F0400202B
:105150008C070020670500208407002080070020BE
:10516000FFFFFBFF302B01D100F008FC0ED8192BFC
:1051700000D16DE101D201F0B0F81A2B01D001F09D
:105180001AFB02AB1A7AE24900234FE1322B01D11C
:1051900000F010FC00D27EE3712B01D001F00BFB7C
:1051A0000420DC4BDC4D1978C9B24A1CD2B21A700B
:1051B000DA4A50541978C9B2481CC0B2187003209A
:1051C00050541978C9B2481CC0B21870002050540D
:1051D0001978C9B2481CC0B218702878C0B2441CF3
:1051E000E4B22C7050541978C9B2481CC0B218707F
:1051F000F12318E10625C7490C78E4B2601CC0B25F
:105200000870C64805550C78E4B2651CEDB20D7007
:10521000052505550D78EDB26C1CE4B20C70002428
:1052200044550D78EDB26E1CF6B20E7044550D78F3
:10523000EDB26E1CF6B20E70812646550D78EDB2B9
:105240006E1CF6B20E70FE2646550D78EDB26E1C41
:10525000F6B20E70AF214155AF49B1480B70B1495C
:105260000C70B1490C70016899430160AF4B1B7819
:10527000A34201D101F09FFA2CE004218020AC4B25
:10528000C0021960A6490B6803430B60A74B1B784B
:10529000002B1FD0A74B1B88C72B1BD88021402475
:1052A000A54883680B438360A4488368A343836055
:1052B0000020A34B1870A34B05301870A24B197037
:1052C0001168A24B0B401360FA22A14B52001A60E6
:1052D00001F071FA80211368C90110E0681EC0B2A4
:1052E0002100FBF7B3FC072D01D001F064FA3E2C3E
:1052F00001D001F060FA8021964A090513680B433A
:10530000136001F058FA0B20824B00251978824E69
:10531000C9B24A1CD2B21A70804A50541978C9B224
:10532000481CC0B218700A2050541978C9B2481CE1
:10533000C0B2187055541978C9B2481CC0B2187060
:105340003078C0B2441CE4B2347050541978C9B2F9
:10535000481CC0B21870842050541978C9B2481C37
:10536000C0B2187057541978C9B2481CC0B218702E
:1053700055541978C9B2481CC0B218703E20505418
:105380001978C9B2481CC0B2187073480468240E5A
:1053900054541C78E4B2611CC9B219700168090C3C
:1053A000C9B211551C78E4B2611CC9B21970016808
:1053B000090AC9B211551978C9B24C1CE4B21C7063
:1053C0000368BBE20520534B534D1978C9B24A1C00
:1053D000D2B21A70514A50541978C9B2481CC0B29E
:1053E0001870042050541978C9B2481CC0B2187003
:1053F000002050541978C9B2481CC0B218702878DF
:10540000C0B2441CE4B22C7050541978C9B2481C84
:10541000C0B21870822050541978C9B2481CC0B26A
:10542000187002AB9B79535401F0C5F9D8B282428F
:1054300005D902AC1819407AC8540133F6E70023A5
:105440008B540421364A02ABDF7113680B4313609F
:1054500002ABD979002900D180E000232C4AD15C2D
:10546000D8B2002903D00133182BF8D11800294BEA
:10547000C41D1978E4B2C9B24A1CD2B21A70274AC4
:1054800054541978C9B24C1CE4B21C70841DE4B2A7
:1054900054541C78E4B2611CC9B219700021115532
:1054A0001C78E4B2651CEDB21D701B4DAC46614624
:1054B0002D78EDB26E1CF6B20E7015551C780021D9
:1054C000E4B2651CEDB21D70952515551C78104E83
:1054D000E4B2651CEDB21D70115500211C78E4B2D8
:1054E000651CEDB21D7017551C78E4B2651CEDB259
:1054F0001D701055CCB2844201D301F05CF91C78C8
:10550000E4B2651CEDB21D70755C01311555F1E713
:105510004E050020EA020020400500203F04002044
:105520008007002084070020670500201603002064
:1055300000E100E07405002000400050C040005031
:1055400072050020B002002076050020FFFFBFDFBB
:10555000E00200206C050020B80200201224F84B65
:10556000F84E1878C0B2421CD2B21A70F64A1454DF
:105570001878C0B2441CE4B21C701124145418787A
:10558000C0B2441CE4B21C7011541878C0B2441C60
:10559000E4B21C703478E4B2651CEDB2357014547A
:1055A0001878C0B2441CE4B21C70952414541878C6
:1055B000C0B2441CE4B21C7011541878C0B2441C30
:1055C000E4B21C7011541978C9B2481CC0B21870EA
:1055D000092050541978C9B2481CC0B21870422032
:1055E00050541978C9B24C1CE4B21C70692454544C
:1055F0001978C9B24D1CEDB21D7044255554197867
:10560000C9B24D1CEDB21D7054541978C9B24C1C6E
:10561000E4B21C7050541978C9B2481CC0B218705A
:105620006F2050541978C9B24C1CE4B21C7050540D
:105630001978C9B2481CC0B2187073205054197838
:10564000C9B2481CC0B21870742050541978C9B23D
:10565000481CC0B21870652050541978C9B2481C53
:10566000C0B218707223DEE60720B54B002519780A
:10567000B44EC9B24A1CD2B21A70B34A5054197807
:10568000C9B2481CC0B21870062050541978C9B26B
:10569000481CC0B2187055541978C9B2481CC0B221
:1056A00018703078C0B2441CE4B234705054197889
:1056B000C9B2481CC0B21870852050541978C9B2BC
:1056C000481CC0B218700A2050541978C9B2481C3E
:1056D000C0B21870575400F090FF80259B4BAD026C
:1056E0001C689B482C4207D01D689A4C2C401C60BB
:1056F0007F230478234005E01C682C431C60802332
:1057000004782343037013788E4DDBB2581CC0B26B
:1057100010700520C8541378DBB2581CC0B210704A
:105720000420C8541378DBB2581CC0B2107000209B
:10573000C8541378DBB2581CC0B210702878C0B2BD
:10574000441CE4B22C70C8541378DBB2581CC0B2AD
:1057500010708720C8541078C0B2431CDBB213709D
:105760007A4B1B685B0C3B400B5401F024F806207D
:10577000734B00241978734EC9B24A1CD2B21A7006
:10578000714A50541978C9B2481CC0B2187005202B
:1057900050541978C9B2481CC0B2187054541978C2
:1057A000C9B2481CC0B218703078C0B2451CEDB206
:1057B000357050541978C9B2481CC0B21870862090
:1057C00050541978C9B2481CC0B218705454197892
:1057D000C9B2481CC0B21870545400F0ECFF052048
:1057E000574B584D1978C9B24A1CD2B21A70564A52
:1057F00050541978C9B2481CC0B2187004205054D3
:105800001978C9B2481CC0B21870002050541978D9
:10581000C9B2481CC0B218702878C0B2441CE4B2A7
:105820002C7050541978C9B2481CC0B21870882026
:1058300000F038FF1378434DDBB2581CC0B2107033
:105840000520C8541378DBB2581CC0B21070042075
:10585000C8541378DBB2581CC0B210700020C85472
:105860001378DBB2581CC0B210702878C0B2441C48
:10587000E4B22C70C8541378DBB2581CC0B210705C
:105880008A20C8541378DBB2581CC0B21070802232
:10589000CA5400F090FF04212F4B304D1960304B5B
:1058A0001F70304B1B88C72B18D840242E487C31E2
:1058B00083680B4383602D488368A3438360002083
:1058C0002B4B1870224B29707B3919701168294BAA
:1058D0000B401360FA22284B52001A600520184B27
:1058E000184E1978C9B24A1CD2B21A70164A5054CE
:1058F0001978C9B2481CC0B21870042050541978E5
:10590000C9B2481CC0B21870002050541978C9B2EE
:10591000481CC0B218703078C0B2441CE4B2347075
:1059200050541978C9B2481CC0B21870B0205054F5
:105930001978C9B2481CC0B218702B78DBB272E576
:10594000EA020020400500203F04002080070020DC
:10595000B0020020FFFFFDFF00E100E0760500201F
:10596000660500207405002000400050C040005033
:1059700072050020FFFFBFDFE00200208020CA493F
:105980008B6883438B60C94940388B6803438B60C5
:105990000023C7490B70C7490878052801D1023098
:1059A00000E006200870C4490B7081211368890546
:1059B0000B4313600F20C14BC14D1978C9B24A1C6B
:1059C000D2B21A70BF4A50541978C9B2481CC0B23A
:1059D0001870042050541878C0B2411CC9B2197014
:1059E000002111541878C0B2441CE4B21C702C7809
:1059F000E4B2661CF6B22E7014541878C0B2441C7F
:105A0000E4B21C70B02414541878C0B2441CE4B240
:105A10001C70A94CA4462478E4B214541878C0B27F
:105A2000441CE4B21C70092414541878C0B2441CFD
:105A3000E4B21C7011541878C0B2441CE4B21C705B
:105A40002C78E4B2661CF6B22E7014541878C0B2EA
:105A5000441CE4B21C70B22414541878C0B2441C24
:105A6000E4B21C7017541878C0B2441CE4B21C7025
:105A70006446247864B28C4204DA93494C780A2153
:105A80006143C9B211541978C9B2481CC0B2187028
:105A9000002050541978C9B24C1CE4B21C70505408
:105AA0001978C9B24C1CE4B21C7002245454197801
:105AB000C9B24C1CE4B21C70505400F07CFE834B05
:105AC0001A687E4B520331D5052019787C4DC9B236
:105AD0004A1CD2B21A707B4A50541978C9B2481C79
:105AE000C0B21870042050541978C9B2481CC0B212
:105AF0001870002050541978C9B2481CC0B21870F0
:105B00002878C0B2441CE4B22C7050541978C9B241
:105B1000481CC0B21870B02050541978C9B2481C43
:105B2000C0B2187064480078C0B25054052019788B
:105B30000025C9B24A1CD2B21A70624A604E505453
:105B40001978C9B2481CC0B2187004205054197892
:105B5000C9B2481CC0B2187055541978C9B2481C53
:105B6000C0B218703078C0B2441CE4B234705054E3
:105B70001978C9B2481CC0B21870922050541978D4
:105B8000C9B2481CC0B2187012235354504B1D7038
:105B900000F011FE02AB9B794D4A152B37D013D87C
:105BA000102B2CD007D80C2B3FD00F2B25D00B2B34
:105BB0003DD10E233AE0122B25D022D3132B24D033
:105BC000142B34D1052331E01A2B26D008D8172BFB
:105BD00021D01ED3182B26D0192B28D10D2325E038
:105BE000FC2B1ED003D81C2B21D110231EE0FD2B33
:105BF00015D0FE2B1BD1112318E0002316E01770DF
:105C000015E0022312E0032310E004230EE0062334
:105C10000CE007230AE0082308E0092306E00A2332
:105C200004E00B2302E00C2300E00F231370062096
:105C30000525224B224E1978C9B24A1CD2B21A70DD
:105C4000204A50541978C9B2481CC0B21870555433
:105C50001978C9B2481CC0B2187000205054197885
:105C6000C9B2481CC0B218703078C0B2441CE4B24B
:105C70003470174C50542178112900D9AFE1080035
:105C800000F0FEFF280036004C00610077008D0018
:105C9000A300B100DE00F4000B0120013501430137
:105CA0005B0169017F01960100400050C040005037
:105CB00066050020B002002076050020EA020020E0
:105CC000400500203F040020EB0200208007002058
:105CD000680200201878C0B2451CEDB21D709025F6
:105CE00015541878C0B2451CEDB21D700F2522E086
:105CF0001878C0B2451CEDB21D7090251554187867
:105D0000C0B2451CEDB21D70102515541878C0B2F4
:105D1000451CEDB21D70E54B5B7847E11878C0B2C9
:105D2000451CEDB21D70902515541878C0B2451C65
:105D3000EDB21D70112515541878C0B2451CEDB296
:105D40001D70175460E11878C0B2451CEDB21D708B
:105D5000902515541878C0B2451CEDB21D7012255F
:105D600015541878C0B2451CEDB21D70CF4B5B794D
:105D7000E1E01878C0B2451CEDB21D7090251554B5
:105D80001878C0B2451CEDB21D7013251554187853
:105D9000C0B2451CEDB21D70C44B9B7806E118786B
:105DA000C0B2451CEDB21D70902515541878C0B2D4
:105DB000451CEDB21D70142515541878C0B2451C51
:105DC000EDB21D70B94BDB78F0E01878C0B2451C1D
:105DD000EDB21D70902515541878C0B2451CEDB277
:105DE0001D701525A7E71878C0B2451CEDB21D70CF
:105DF000902515541878C0B2451CEDB21D701625BB
:105E00001554AA480079C0B203280BD0042810D03A
:105E1000022800D0F8E01878C0B2451CEDB21D7021
:105E20008B23F0E01878C0B2451CEDB21D709B23A7
:105E3000E9E01878C0B2451CEDB21D70AA23E2E07B
:105E40001878C0B2451CEDB21D7090251554187815
:105E5000C0B2451CEDB21D70172515541878C0B29C
:105E6000451CEDB21D70914B9B799FE01878C0B234
:105E7000451CEDB21D70902515541878C0B2451C14
:105E8000EDB21D701A2515541878C0B2451CEDB23C
:105E90001D70864B5B795B084DE01878C0B2451CDD
:105EA000EDB21D70902515541878C0B2451CEDB2A6
:105EB0001D70FD2515541878C0B2451CEDB21D703B
:105EC0000823A0E01878C0B2451CEDB21D709025E3
:105ED00015541878C0B2451CEDB21D70FC25155440
:105EE0001878C0B2451CEDB21D7018238BE01878ED
:105EF000C0B2451CEDB21D70902515541878C0B283
:105F0000451CEDB21D70182515E71878C0B2451C68
:105F1000EDB21D70902515541878C0B2451CEDB235
:105F20001D70192515541878C0B2451CEDB21D70AE
:105F30005E4B5B799B093B4065E01878C0B2451C1D
:105F4000EDB21D70902515541878C0B2451CEDB205
:105F50001D700B2539E01878C0B2451CEDB21D70DC
:105F6000902515541878C0B2451CEDB21D700C2553
:105F700015541878C0B2451CEDB21D704B4BDB7C3C
:105F800014E01878C0B2451CEDB21D709025155470
:105F90001878C0B2451CEDB21D701C251554187838
:105FA000C0B2451CEDB21D70404B9B7CDBB22AE0B9
:105FB0001878C0B2451CEDB21D70902515541878A4
:105FC000C0B2451CEDB21D70FE2515541878C0B244
:105FD000451CEDB21D70354B5B79DB0913E0187879
:105FE0000438155404251878033815541878C0B2AD
:105FF000451CEDB21D70912515541878C0B2451C92
:10600000EDB21D70FF23135401312170D3E3284CEE
:10601000284D23780020DBB25A1CD2B2227006220F
:10602000EA542378244EDBB25A1CD2B222700522E5
:10603000EA542378DBB25A1CD2B22270E854237897
:10604000DBB25A1CD2B222703278D2B2511CC9B221
:106050003170EA542378DBB25A1CD2B222709022FB
:10606000EA542278D2B2531CDBB2237002AB9B7984
:10607000AB54142B5CD035D8102B00D1AEE01DD81A
:106080000B2B00D1E3E00C2B00D01EE12378122073
:10609000DBB25A1CD2B2227002AAD4792100EC548D
:1060A000FAF7D4FD014BDC7485E3C046EB02002017
:1060B000EA0200203F04002040050020122B24D0DB
:1060C000132B00D001E123780120DBB25A1CD2B29D
:1060D000227002AAD4792100EC54FAF7B7FDDA4B0A
:1060E0009C7068E3192B00D198E004D8162B35D0AA
:1060F000172B5DD0E9E01C2B00D1C1E0FE2B00D1B5
:10610000CDE01A2B00D0E0E076E0CF4E02AA737902
:10611000D0792278DBB2D2B2511CC9B221700028EA
:1061200002D0AF543B4301E0A854BB431C00A1E0A4
:1061300002ABDB79FA2B02D9FA2302AAD3712378B6
:106140000220DBB25A1CD2B2227002AAD4792100FA
:10615000EC54FAF77BFDBC4BDC702CE302ABDB7933
:10616000B94EAA2B08D9AA2302AA04210320D3716D
:10617000FAF76CFD042312E09A2B08D88B2302AAAD
:1061800002210320D371FAF761FD022307E0032106
:106190009B2302AA0800D371FAF758FD0323337139
:1061A0002378DBB25A1CD2B2227002AAD27992E0D2
:1061B00002ABDB79632B02D8002302AAD3712378C8
:1061C0000520DBB25A1CD2B2227002AAD479210077
:1061D000EC54FAF73BFD9C4B9C71ECE22378DBB26C
:1061E0005A1CD2B2227002AAD4792100EC54FAF7D8
:1061F0002DFD954B5C70DEE2934E02AA7379D07947
:106200002278DBB2D2B2511CC9B22170002802D070
:10621000AF54022429E0A854022216E08A4E02AAB2
:106220007379D279DBB2002A07D02278D2B2511C1E
:10623000C9B22170AF54402417E02278D2B2511C69
:10624000C9B221700021A954402293436EE77E4ECB
:1062500002AA7379D0792278DBB2D2B2511CC9B2CA
:106260002170002803D08024AF541C4302E07F2417
:10627000A8541C4021000420FAF7E8FC74719AE24B
:1062800023781120DBB25A1CD2B2227002AAD47930
:106290002100EC54FAF7DAFC6B4B9C748BE2227809
:1062A0000420D2B2531CDBB2237002ABDB79AB54B7
:1062B0007F22654D6C7914405A1E9341DB011C43CB
:1062C0002100FAF7C3FC6C7175E22378DBB25A1C2B
:1062D000D2B222700022EA546DE202AB9A795B4B93
:1062E0001A7002AAD2795A7002AA127A9A7002AA75
:1062F000527ADA705FE202AB9A79092A05D802A8CD
:106300001318DB799C46092B08D90A68504B1340B7
:106310000B600A684F4B13400B60D1E34E4B1C7867
:10632000E4B2611CC9B2197061465018C0B24B4941
:10633000851DEDB20D551C780530E4B2651CEDB23B
:10634000C0B21D7008551C78E4B2601CC0B2187051
:10635000002008551C784248E4B2651CEDB21D705F
:106360003F4D2D78EDB26E1CF6B206700D551C78BF
:106370000020E4B2651CEDB21D7093250D551C780C
:106380000090E4B2651CEDB21D700A551C00684611
:106390000578AA420ED9257802A8EDB26E1CF6B295
:1063A0002670009E3618F6792C4846550098013024
:1063B0000090ECE71878C0B2451CEDB21D70634642
:1063C0000B540023D9B28C450CD9217802ADC9B247
:1063D000481CC0B2207098184019007A1F4D013334
:1063E0006854EFE702ABDD790A210023303DEDB2BE
:1063F0000133D8B2824207D902AC4D431819C07993
:1064000030382D18EDB2F3E702A953180A20002105
:106410001C7A303CE4B20131CBB29C4501D8FEF786
:106420005DFF8B1802AE44439B191B7A303BE41886
:10643000E4B2F0E702AB9979092913D91168044B4A
:106440000B40136038E3C046EB020020E602002058
:10645000FFFFFFFDFFFFFFFBEA0200203F040020DB
:106460004005002000220A2002ABDB79303BDBB282
:1064700000930132D3B299420AD902AC1319DC79E4
:10648000009D23004543303BEB18DBB20093F0E75F
:10649000009B072B02D10A22E74BDA710800E74C78
:1064A00009302278C0B2D2B2531CDBB22370E44B65
:1064B00098542278D2B2501CC0B220700800083024
:1064C000C0B298542078C0B2421CD2B222700022CE
:1064D0001A542078C0B2451CEDB22570D94DAC4697
:1064E00062462D789C46EDB26E1CF6B216701D54B5
:1064F00020780022C0B2451CEDB2257093252600FD
:106500001D542078C0B2451CEDB225701954D0B28C
:1065100088420BD2307802ABC0B2451CEDB2357068
:10652000D5186346ED7901321D54F0E72378C44D48
:10653000DBB25A1CD2B222700322EA542678009AA7
:10654000F6B2731CDBB22370BB4B6421985CC0B203
:1065500000F0A0FB3030009AB74BC0B2A855985C51
:106560006421C0B200F01CFC2678CBB2F6B20093D6
:10657000731CDBB223700A21009800F08BFB3030D3
:10658000C0B2A85526780A21F6B2731CDBB223707C
:10659000009800F005FC3031C9B2A9550BE1052087
:1065A0001168A94B00250B401360A44BA54E197828
:1065B000C9B24A1CD2B21A70A14A50541978C9B251
:1065C000481CC0B21870042050541978C9B2481C35
:1065D000C0B2187055541978C9B2481CC0B21870AE
:1065E0003078C0B2441CE4B2347050541978C9B247
:1065F000481CC0B21870942050541978C9B2481C75
:10660000C0B218705554D6E0904802A90368497A80
:106610001B0E994200D0CEE002AB9C7AFF230168AA
:10662000090C19408C4200D0C5E0016802ACE47A44
:10663000090A19408C4200D0BDE002A90068097B1C
:106640000340994200D0B6E08021052013688904F8
:106650000B431360794B7B4D1978C9B24A1CD2B2F7
:106660001A70774A50541978C9B2481CC0B21870D1
:10667000042050541978C9B2481CC0B218700020C8
:1066800050541978C9B2481CC0B218702878C0B2EA
:10669000441CE4B22C7050541978C9B2481CC0B2E2
:1066A0001870942050541978C9B2481CC0B21870A0
:1066B000575480E002AB9B79002B7CD102AB5B7A14
:1066C0003E2B78D1614902AA0B68927A1B0E9A423E
:1066D00071D102ABD87AFF230A68120C1A4090429B
:1066E00069D10A6802A8007B120A1A40904262D15E
:1066F00002AA0968527B0B409A425CD1FAF798FAD9
:10670000FAF77EFAF8204002FAF750FA2378504A56
:10671000504C1B021343236021684F48FAF7EEF9EF
:1067200003214E4A13680B432360236813604C4ACD
:106730004C4B1A60FEE780204B498B6883438B608B
:106740004A4940388B6803438B60FA21484B8900E3
:10675000198000218120474B80051970136803437D
:106760001360454A454B1068034090201360444A2B
:106770009368034393608022424B9201DA67424B55
:10678000424A1970424BFF311A60424A11701A682E
:10679000002AFCD12B4B1A70FAF74AFA03212F4A30
:1067A00013680B4313602E4A2E4B1A60A022D205A9
:1067B00093683B43936002AB9B78002B00D063E16E
:1067C00002AA1279092A00D1F9E00AD8032A00D1D5
:1067D0002CE1042A00D057E1274A284B11680B40CE
:1067E00051E1302A00D19BE0312A00D04CE1042154
:1067F000294A204C1160294A1770294A1188294AD0
:10680000C72957D880204026174DA9680143A960A1
:10681000164DA968B143A96023490B700521234B8C
:10682000197020701168224B0B401360FA22184B2C
:1068300052001A6043E0C046EB020020EA0200204A
:106840003F04002040050020FFFFFFFDB8020020AC
:106850003E00FFFFD00200201CF0010000C00050ED
:106860000400FA050CED00E000400050C04000506C
:10687000E40200207605002080070020FFFFFBFFD8
:106880008040005004E100E094070020DC05000097
:10689000E00200203D04002000E100E06605002049
:1068A000740500206C05002072050020B002002055
:1068B000FFFFBFDF80211368C9010B431360052070
:1068C000804B814E1978C9B24A1CD2B21A707F4AE5
:1068D00050541978C9B2481CC0B2187004205054E2
:1068E0001978C9B2481CC0B21870002050541978E9
:1068F000C9B2481CC0B218703078C0B2451CEDB2A5
:10690000357050541978C9B2481CC0B21870B02004
:1069100050541978C9B2481CC0B2187023784BE0A3
:1069200080206B498A6882438A606A4940388A6855
:1069300002438A60684A1370684B1A78052A01D1AD
:10694000023200E00622002081210524644D1A70E5
:10695000644A2870136889050B431360594B5A4EDB
:106960001978C9B24A1CD2B21A70584A54541978CC
:10697000C9B24C1CE4B21C70042454541978C9B236
:106980004C1CE4B21C7050541978C9B2481CC0B2F7
:1069900018703078C0B2441CE4B234705054197886
:1069A000C9B2481CC0B21870B02050541978C9B28E
:1069B000481CC0B218702B78DBB2535464E08020BE
:1069C00043498A6882438A60424940388A68024360
:1069D0008A60FA218120444A89001180404A414955
:1069E00013700A68800502430A6080213F4A8901CA
:1069F000D167FF213E4A13703E4A3F4B1A603F4A1F
:106A000011701A68002AFCD12F4B1A70FAF710F98E
:106A100003213B4A13680B4313603A4A3A4B1A600E
:106A2000A022D20593683B4393602DE08020374934
:106A3000C0020A6802430A60354A1178294A0029CF
:106A40001DD034490988C72919D880204025204CF9
:106A5000A1680143A1601F4CA168A943A1602E4910
:106A60000B7005211D4B19701D4B187011682B4BB5
:106A70000B401360FA22204B52001A6004E0802180
:106A80001368C9010B43136002AB1A785B780133BA
:106A90009A4210DDDBB2D21A02A90A70002201323A
:106AA0000198D1B2884201D8FEF75DFA02A8191800
:106AB000895C8154F3E70B4A1168194B0B40136052
:106AC00013B0F0BDEA020020400500203F04002082
:106AD00000400050C040005066050020B002002079
:106AE000760500206C050020E402002004E100E0AF
:106AF00094070020DC050000E00200203D04002097
:106B000000C000500400FA050CED00E080070020F2
:106B1000160300207405002072050020FFFFBFDF70
:106B2000FFFFFFFBF7B508AC247880250194A02473
:106B3000E405E7686D052F43E760E668204F3740BE
:106B4000E760204C03273B409F0063690C26B3435A
:106B50003B436361019F1C4B3E04A7693B403343A9
:106B6000A361A3681D43194BA5601C6A01252C4332
:106B70001C621C6A002802D11548204002E08020D7
:106B8000C000204318620C20002902D1196A8143F9
:106B900005E0012905D1196A8143042001431962E6
:106BA00008E0022903D1196A81430820F6E7196A2F
:106BB00008431862596AFF2081430A435A62F7BDAD
:106BC000FFFFFFEF00020050FFFF00FF00000E403C
:106BD000FFFBFFFF10B5194C236BDA070CD5184AE1
:106BE0001368002B01D050689847164B07211A688C
:106BF0008A4301210A431A60236B9A070CD5104A75
:106C00001369002B01D0906898470E4B07211A6832
:106C10008A4302210A431A60236B5A070CD5084A9B
:106C20005369002B01D0D0689847064B07211A689A
:106C30008A4304210A431A6010BDC04600000E407A
:106C40008C02002030000E40064B07211A688A4350
:106C500001210A431A60044B8022196A12010A4377
:106C60001A62704730000E4000000E4002B47146B8
:106C700049084900095C49008E4402BC7047C0467F
:106C800003B47146490840004900095A49008E443E
:106C900003BC7047002243088B4274D303098B4224
:106CA0005FD3030A8B4244D3030B8B4228D3030CDC
:106CB0008B420DD3FF22090212BA030C8B4202D37E
:106CC0001212090265D0030B8B4219D300E0090AA6
:106CD000C30B8B4201D3CB03C01A5241830B8B42AF
:106CE00001D38B03C01A5241430B8B4201D34B0398
:106CF000C01A5241030B8B4201D30B03C01A5241FD
:106D0000C30A8B4201D3CB02C01A5241830A8B4281
:106D100001D38B02C01A5241430A8B4201D34B026A
:106D2000C01A5241030A8B4201D30B02C01A5241CE
:106D3000CDD2C3098B4201D3CB01C01A5241830982
:106D40008B4201D38B01C01A524143098B4201D3BC
:106D50004B01C01A524103098B4201D30B01C01AE7
:106D60005241C3088B4201D3CB00C01A5241830861
:106D70008B4201D38B00C01A524143088B4201D38E
:106D80004B00C01A5241411A00D2014652411046EE
:106D90007047FFE701B5002000F0F0F802BDC046E3
:106DA0000029F7D076E7704703460B437FD40022D3
:106DB00043088B4274D303098B425FD3030A8B428F
:106DC00044D3030B8B4228D3030C8B420DD3FF22F9
:106DD000090212BA030C8B4202D31212090265D0C7
:106DE000030B8B4219D300E0090AC30B8B4201D37A
:106DF000CB03C01A5241830B8B4201D38B03C01AC1
:106E00005241430B8B4201D34B03C01A5241030B37
:106E10008B4201D30B03C01A5241C30A8B4201D3E8
:106E2000CB02C01A5241830A8B4201D38B02C01A93
:106E30005241430A8B4201D34B02C01A5241030A0A
:106E40008B4201D30B02C01A5241CDD2C3098B42EF
:106E500001D3CB01C01A524183098B4201D38B016C
:106E6000C01A524143098B4201D34B01C01A52410F
:106E700003098B4201D30B01C01A5241C3088B4254
:106E800001D3CB00C01A524183088B4201D38B003F
:106E9000C01A524143088B4201D34B00C01A5241E1
:106EA000411A00D201465241104670475DE0CA0FB8
:106EB00000D04942031000D34042534000229C4678
:106EC00003098B422DD3030A8B4212D3FC22890182
:106ED00012BA030A8B420CD3890192118B4208D358
:106EE000890192118B4204D389013AD0921100E0BA
:106EF0008909C3098B4201D3CB01C01A52418309CE
:106F00008B4201D38B01C01A524143098B4201D3FA
:106F10004B01C01A524103098B4201D30B01C01A25
:106F20005241C3088B4201D3CB00C01A524183089F
:106F30008B4201D38B00C01A5241D9D243088B42F5
:106F400001D34B00C01A5241411A00D20146634698
:106F500052415B10104601D34042002B00D54942FC
:106F6000704763465B1000D3404201B5002000F03B
:106F700005F802BD0029F8D016E770477047C046F3
:106F800000000000200000000000100020001000A1
:106F900030353A3F44494E54585C61666B7075A574
:106FA0001264640381C80A3E041EFFFFFFFFFFFF57
:106FB000FF0530FF0204081001000000020000007D
:086FC0000200000004000000C3
:106FC800FF40404040404040334040403440353628
:106FD80040404040404040403A4040403B403C37C1
:106FE800404040403F403D3840403E3940FB4040F3
:106FF80040404040404040402440404023402221FF
:10700800404040401F401E2040401D1C401B404047
:10701800404040401940181A40401716401540405B
:1070280040402514401340404032404040404040DA
:107038004040404040404040FE4040400E400D0C23
:10704800404040400A40090B404008074006404085
:107058004040404004400305404002014000404099
:1070680040400F10401140404012404040404040D6
:1070780040404040FD402B3040402A2F40314040A6
:107088004040292E402D4040402C40404040404048
:107098004040FA2840274040402640404040404079
:1070A80040FC0000001BB7000000000000805101F8
:1070B80010270000008051010080510116000000D7
:00000001FF
